:020000040000FA
:0C000000000000000FEF10F0FCEF40F0DB
:08001800C8EF41F0800E016EFB
:10002000FE0EA9D9010EA7D9750E146E300E22EF5F
:1000300002F0016A018E236EFE0E9DD923509BD1E2
:10004000076A800E3A6E00D01B6A1C6A1D6A1E6A1F
:10005000099A9CD9D8A01200D30FD8B4098A2D0FC1
:10006000C60FF7E20A0FF5E3176E166A156A146AEF
:100070000A0E136EB3EC02F0175013241B6E1450CB
:100080001C6E000ED8B0010E1C2615501D6E000E01
:10009000D8B0010E1D2616501E6E000ED8B0010EEF
:1000A0001E26070607E072D9D8A01200C60F02E28A
:1000B0000A0FDAE209AA0BD01B1E1C1E1D1E1E1EF3
:1000C0001B2AD8B41C2AD8B41D2AD8B41E2A1B5007
:1000D000D880120030D803D0076A1B6E1C6A0096C5
:1000E0000750D8B40086050E066E270E186E100E47
:1000F0000CD8030E186EE80E08D8186A640E05D8DE
:10010000186A0A0E02D81B5007D0176E1C50146EC6
:100110001B50136ED6D91350136E064E009607501F
:1001200002E0065C07E21350D8A4009600B602D0A5
:10013000300F21D112001CAE12001B501C10D8B47D
:1001400012001B1E1C1E1B4A1C2A2D0E14D13C6EB5
:1001500027AE02D02D0E0FD9293E04D0283E02D062
:10016000274A272A326A336A346A356A278E6A0E2A
:100170002626D8902732283229323532343233328B
:100180003232263EF6D72950265C2926265E285094
:10019000275C2826275E076A38D82E0EECD83D6AE1
:1001A000D8903234296E3334286E3434276E353487
:1001B000266E3D36D89029362836273626363D36E7
:1001C000325029263350D8B0333C28263450D8B08A
:1001D000343C27263550D8B0353C2626D8B03D3E95
:1001E000D89029362836273626363D363D50300FF2
:1001F000C2D829C032F028C033F027C034F026C05E
:1002000035F03C2ECCD7D89012000096075003E171
:1002100000860A0E076E29C016F028C015F027C008
:1002200014F026C013F0066A1E6A1D6A1C6A0A0EC4
:100230001B6E1CD9062A0650075CF6E11B50D8A499
:10024000009600A602D0072C03D01B50300F93D885
:10025000072EE1D712001B6E0650D8B412001BC047
:10026000E9FF1CC0EAFFEF50D8B4120084D81B4A43
:100270001C2A0606F1D7A66AA68E0900F55002E0F0
:1002800002D8FBD71200206E8998899A9298929A88
:10029000F00E9216205000B21ED03A0E146E980E38
:1002A000D1D8330E1F6E29D8130E146E880ECAD8FB
:1002B00024D8640EC6D821D8640EC3D8220E1F6E6F
:1002C0001CD8280E07D80C0E05D8060E03D80082BD
:1002D000205001D000801F6E00A009D0899A030829
:1002E0000AE309D8090E146EC40EACD812000080BF
:1002F000FE0814E0898A1F3A00A000908988F00E59
:1003000080161F500F0B8012000000D089981F3AF2
:10031000000000D000B0F1D7320E93D82050120068
:1003200002C013F008C014F0176A186A000000D069
:1003300000009EBA11D0E868172618221322142252
:10034000D8A012001748183CF1D7E80E176E010E1E
:10035000186EEED79EAAFED7AE50D8801200A66ABD
:10036000A68E0900F55002E002D8FBD712009EA825
:10037000FED7AD6E120001BE86D701B4F8D701A238
:1003800005D001B003D001B2EE6E12003AAE03D038
:10039000EE50D88012003A52C3E03A04DBE0A86E77
:1003A000F2CFF3FFF29EA66AA684550EA76EAA0EA0
:1003B000A76EA682A6B2FED7A694A94AAA2AF3BE21
:1003C000F28EA68E1200A96EA66AA680A850A94A2F
:1003D000AA2AA68E1200080E1F6EEA6803C0E9FF63
:1003E000045009B419D909A419D9E26803C0E1FF7E
:1003F0000250120FE96E081CEF161F500EE009B0F4
:10040000F3D802C0E9FF14321332EF500810D8A01D
:100410000818EF6E03D81F2EF6D712000450E71A03
:10042000000000D0E71A1200186A176EFF0E172698
:10043000182200D0D8A01200030E146EE60E02D8C7
:10044000F5D7146AFD0F136E01D01306000000D01B
:10045000E86A145AFAE21200010F206E0A0E176EB3
:10046000186A2FD8202EFDD71B5012002E6A2F6A33
:10047000306A316A210E196E15D02E362F3630367D
:1004800031361B502E5C1C502F581D5030581E50BA
:10049000315808E3316E1B502E5E1C502F5A1D50F0
:1004A000305AD8801336143615361636192EE5D73D
:1004B00031C01EF030C01DF02FC01CF02E501B6E3E
:1004C00012001C6A1B6A100EF36E14341B361C36A5
:1004D00017501B5C18501C5805E317501B5E185032
:1004E0001C5AD88013361436F32EEFD7135012004F
:1004F00022501C18800BF46E22AE05D0211E221E45
:10050000212AD8B4222A1CAE05D01B1E1C1E1B2A71
:10051000D8B41C2A176A136A146A186A1C5002E1BC
:100520001B5018E0100EF36ED89021362236173685
:1005300018361C50185C02E11B50175C07E31B5077
:10054000175ED8A018061C50185ED88013361436D3
:10055000F32EEAD7F4AE05D0131E141E132AD8B416
:10056000142A1350120016C031F015C030F014C018
:100570002FF013C02EF030501B02F3CF15F0F4CF44
:1005800016F02F501C02F3501526F45016222E5050
:100590001D02F3501526F450162231501B02F35061
:1005A000162630501C02F35016262F501D02F35011
:1005B00016262E501E02F35016262E501B02F3CF85
:1005C00013F0F4CF14F02F501B02F3501426F45004
:1005D0001522000E16222E501C02F3501426F45041
:1005E0001522000E16221200176A186A04D014325F
:1005F000133217361836FF0FFAE218C014F01750EE
:10060000136E1200136E14BE02D813501200131E84
:10061000141E134A142A1200EF1203D0FF0AEF1619
:1006200001D0FF0AE988E92AEC161200FE0EDBCFA2
:10063000E6FFFF0EDBCFE6FFDD52DD521200A66AB9
:10064000A68E0900F55002E0EE6EFBD71200E752CD
:10065000E6CFEEFF02E0E82EFAD71200F34E02D00A
:10066000E652FCD7E6CFEEFFE82EFCD71200E46698
:10067000FED7F36EE552F32EFDD7E6CFEEFFE82E60
:10068000FCD71200A66AA68EEE500900F55C02E1C6
:10069000F566FAD71200A66AA68EEE500900F55C40
:1006A00003E1F566FAD7010C000CA66AA68EEE509F
:1006B0000900F55C03E1F566FAD7000C010C316A1C
:1006C00035C016F034C015F033C014F03250136E3C
:1006D00005E033AE03D03180800E141A14BE21D051
:1006E000010E165C000E1558000E14587F0E13589C
:1006F00018E3356A346A336A7F0E326E16C039F0F9
:1007000015C038F014C037F013C036F002EC08F012
:1007100035C016F034C015F033C014F032C013F0F9
:1007200031820A0E356E890E346E340E336E7C0EB5
:10073000326E16C039F015C038F014C037F013C04F
:1007400036F068EC08F016C039F015C038F014C067
:1007500037F013C036F068EC08F07C0E396E790E75
:10076000386E350E376E810E366E74EC07F016C09B
:1007700039F015C038F014C037F013C036F068EC0B
:1007800008F016C039F015C038F014C037F013C0A7
:1007900036F068EC08F03F0E396E020E386E330EFC
:1007A000376E830E366E74EC07F016C039F015C044
:1007B00038F014C037F013C036F068EC08F016C0FB
:1007C00039F015C038F014C037F013C036F068ECBB
:1007D00008F0330E396E8C0E386E1E0E376E830E97
:1007E000366E74EC07F035C01AF034C019F033C01F
:1007F00018F032C017F01650356E1550346E145084
:10080000336E1350326E16C039F015C038F014C074
:1008100037F013C036F068EC08F01B0E396EE40EAA
:10082000386E350E376E820E366E74EC07F016C0D9
:1008300039F015C038F014C037F013C036F068EC4A
:1008400008F016C039F015C038F014C037F013C0E6
:1008500036F068EC08F0A40E396EDB0E386E670EC9
:10086000376E830E366E74EC07F016C039F015C083
:1008700038F014C037F013C036F068EC08F016C03A
:1008800039F015C038F014C037F013C036F068ECFA
:1008900008F0330E396E8C0E386E1E0E376E830ED6
:1008A000366E74EC07F035C01EF034C01DF033C056
:1008B0001CF032C01BF016C035F015C034F014C067
:1008C00033F013C032F01AC039F019C038F018C034
:1008D00037F017C036F068EC08F01EC039F01DC0C4
:1008E00038F01CC037F01BC036F002EC08F035C001
:1008F00039F034C038F033C037F032C036F031A2AE
:100900000AD0DB0E356E0F0E346E490E336E7F0E3D
:10091000326E72EC07F031A002D0800E331A3550DF
:100920001200010E1B6E3EC01DF03E8C1E6A1B663F
:1009300002D033BE1E8E339E880E32603E8A35C092
:1009400013F034C014F033C015F032C016F0830E2B
:10095000396EF90E386E220E376E7F0E366E68ECE9
:1009600008F0B6EC08F032A004D0322A000E332290
:100970003422070E32141C6E030E1C6404D0800E49
:100980001E1A040E1C5E356A15EC09F032501A6E00
:100990006DE035C017F034C018F033C019F0396A73
:1009A0000F0E386EC90E376E7E0E366E68EC08F08C
:1009B00013C039F014C038F015C037F016C036F047
:1009C00074EC07F035C013F034C014F033C015F0E8
:1009D00032C016F017C035F018C034F019C033F02B
:1009E0001AC032F0396AA20E386EDA0E376E6E0E09
:1009F000366E68EC08F013C039F014C038F015C03A
:100A000037F016C036F074EC07F035C013F034C080
:100A100014F033C015F032C016F017C035F018C00E
:100A200034F019C033F01AC032F0200E396EA20E25
:100A3000386E850E376E5C0E366E68EC08F013C0AB
:100A400039F014C038F015C037F016C036F074EC29
:100A500007F03250166E366E3350156E376E3450C6
:100A6000146E386E3550136E396E0CD01650326ECF
:100A7000366E1550336E376E1450346E386E135018
:100A8000356E396E68EC08F035C017F034C018F0D8
:100A900033C019F032C01AF01C301C18010B1B189F
:100AA0004EE0CE0E396EF50E386E4C0E376E6F0E70
:100AB000366E68EC08F01A0E396E060E386EB60EF9
:100AC000376E750E366E74EC07F017C039F018C02B
:100AD00038F019C037F01AC036F068EC08F0A50EEF
:100AE000396EAA0E386E2A0E376E7A0E366EFCD923
:100AF00017C039F018C038F019C037F01AC036F0F6
:100B000068EC08F017C039F018C038F019C037F099
:100B10001AC036F068EC08F017C039F018C038F089
:100B200019C037F01AC036F036663606DBD93E9C5F
:100B3000396A386A376A7F0E366ED6D956D0F90EC2
:100B4000396E680E386E360E376E6C0E366E68EC87
:100B500008F0C00E396E070E386ED00E376E720E6A
:100B6000366EC2D917C039F018C038F019C037F046
:100B70001AC036F068EC08F0840E396E880E386EB4
:100B8000080E376E780E366EAFD917C039F018C020
:100B900038F019C037F01AC036F068EC08F0AB0E28
:100BA000396EAA0E386E376E7C0E366E9DD917C020
:100BB00039F018C038F019C037F01AC036F068ECB8
:100BC00008F013C039F014C038F015C037F016C063
:100BD00036F068EC08F03E9C13C039F014C038F0D1
:100BE00015C037F016C036F07FD9800E1B5202E0D8
:100BF0001CB21E1A1EBE331A1DBC3E8C355012008C
:100C000033BEA6D03252D8B4A4D032C01CF03EC0FD
:100C10001DF03E8C7F0E326E396A386A376A366E46
:100C200061D935C013F034C014F033C015F032C0B0
:100C300016F0130E396ECB0E386E030E376E840E1F
:100C4000366E52D913C039F014C038F015C037F0E1
:100C500016C036F068EC08F0BC0E396E5A0E386ECD
:100C6000050E376E860E366E3FD913C039F014C0AC
:100C700038F015C037F016C036F068EC08F0830E77
:100C8000396E300E386E720E376E850E366E2CD978
:100C900035C017F034C018F033C019F032C01AF064
:100CA00013C035F014C034F015C033F016C032F064
:100CB0008E0E396ED70E386E6B0E376E810E366E15
:100CC00068EC08F0B50E396E290E386E4E0E376E90
:100CD000840E366E09D913C039F014C038F015C02F
:100CE00037F016C036F0F4D9800E396E300E386EFB
:100CF000720E376E840E366EF7D817C039F018C0F2
:100D000038F019C037F01AC036F07CD913C039F06A
:100D100014C038F015C037F016C036F0D9D9396A8A
:100D2000386A376A7F0E366EDFD81CB009D0F30EF2
:100D3000396E040E386E350E376E7F0E366EC8D99A
:100D40007F0E1C261C30326E1DBC03D03E9C01D091
:100D50003E8A3550120032503662000C33503762F2
:100D6000000C34503862000C35503962000C010C14
:100D700037503318416E41BE30D037BE17D0365091
:100D8000325CD8A0000CD8A4010C3750335CD8A03A
:100D9000000CD8A4010C3850345CD8A0000CD8A4A6
:100DA000010C3950355CD8A0000C010C3250365C77
:100DB000D8A0000CD8A4010C3350375CD8A0000C8C
:100DC000D8A4010C3450385CD8A0000CD8A4010C75
:100DD0003550395CD8A0000C010C33AE010C000C6E
:100DE00037503318416E41BE34D037BE19D036501B
:100DF000325CD8A0000CD8A4010C3750335CD8A0CA
:100E0000000CD8A4010C3850345CD8A0000CD8A435
:100E1000010C3950355CD8A0000CD8A4010C000C92
:100E20003250365CD8A0000CD8A4010C3350375C8B
:100E3000D8A0000CD8A4010C3450385CD8A0000C09
:100E4000D8A4010C3550395CD8A0000CD8A4010CF2
:100E5000000C33AE010C000C33503718416E41BE0C
:100E600034D033BE19D03250365CD8A0000CD8A490
:100E7000010C3350375CD8A0000CD8A4010C3450BE
:100E8000385CD8A0000CD8A4010C3550395CD8A02F
:100E9000000CD8A4010C000C3650325CD8A0000C19
:100EA000D8A4010C3750335CD8A0000CD8A4010C96
:100EB0003850345CD8A0000CD8A4010C3950355CF3
:100EC000D8A0000CD8A4010C000C37AE010C000C0B
:100ED000396A386A7E0E366E800E33AE000E376E7B
:100EE00003D844D1800E371A3650325C3D6E11E281
:100EF0003D6C325036C032F0366E335037C033F06E
:100F0000376E345038C034F0386E355039C035F053
:100F1000396E1A0E3D6074D0365272E03C6A33501E
:100F2000406E37183F6E338E378E080E3D5E08E3F5
:100F300039C03CF038C039F037C038F0376AF5D7DF
:100F40003D2607E0D8903732383239323C323D2ED8
:100F5000F9D73FAE33D03950355E3850345A375018
:100F6000335A07E2D880000E355634563356800E79
:100F7000401A3C6C04E03506000E345A335A040E15
:100F80003D6E33660DD034C033F035C034F03CC014
:100F900035F03C6A080E325E29E33D2EF2D726D0AA
:100FA00033BE08D0D8903C36353634363336322E00
:100FB000F7D71CD03CAE22D03C6A0FD03950352632
:100FC000385034223750332206E33332343235324C
:100FD0003C32324A0DD03CAE11D0353E0FD0343EBB
:100FE0000DD0333E0BD0D8803590EFD7326A02D087
:100FF0003E823268356A346A800E336E40AE339E6C
:10100000355012003350306E37183F6E365051E075
:10101000325252E0325E7F0E03E2322603E24BD0C0
:1010200032264CE235C02EF034C02FF0308E378E91
:10103000180E406E356A346A336A0BD039502E5C14
:1010400038502F5811E32F6E306A39502E5E0BD076
:1010500004E23750305CF2E007E339502E5E38503E
:101060002F5A3750305AD8803536343633362E36EC
:101070002F363036402EECD733BE07D032521BE02D
:101080003F323206402A3F36E3D707E239502E5E20
:1010900038502F5A3750305A17E3353E15D0343E6A
:1010A00013D0333E11D0333234323532323E0CD08D
:1010B00005D03E8604D03E84326A02D03E82326839
:1010C000356A346A800E336E3FAE339E355012005F
:1010D0003350306E37183F6E3250D8A436503AE055
:1010E00032267E0E03E3325E03E336D0325E31E316
:1010F00035C02EF034C02FF0308E378E356A346A0A
:10110000336A180E406E30322F322E3206E33950D9
:101110003526385034223750332233323432353288
:10112000402EF1D733BE07D03536343633363252FF
:1011300010E03206303416E3353E14D0343E12D07F
:10114000333E10D0D880333234323532323E0AD07A
:1011500003D03E84326A02D03E823268356A346AF5
:10116000800E336E3FAE339E3550120032C040F0D9
:10117000335035C033F0356E3536403235323E6A45
:101180003536403602E33E843E7E06E13E80406ACC
:10119000356A346A336A0BD0402803E0D880353290
:1011A00006D0D890353202E13E8201D03E863EB66E
:1011B00004D03EA20FD03EB407D07F0E356EFF0E96
:1011C000346E336E326E23D0800E356E01D0356AA8
:1011D000000EF6D73EB0FBD7326A9F0E4060EBD7C9
:1011E0007E0E4064F4D79E0E405C07E0D890353206
:1011F000343233323232402AF6D73EA408D0D88077
:10120000000E325633563456355635AEE0D732508E
:101210001200000E33BEFF0E346E356E06D0326EF5
:10122000336A346A356A3F9E0AD03F9E35AE07D096
:10123000D880000E32563356345635563F8E960EB1
:10124000406E355209E0080E402633C032F034C0FB
:1012500033F035C034F011D034520FE1080E405E47
:10126000335007E1080E405E325002E1355010D095
:10127000326A346E32C033F0326A34BE06D0D8904F
:101280003236333634364006F8D73FAE349E4050BF
:1012900032C035F0326E345033C034F0336E120049
:1012A0002020202050494331384634353235202023
:1012B00020202020000020202020416E74656E6ECA
:1012C0006120526F746F72202020000020436F6EE7
:1012D00074726F6C6C6572207665722E0000416EC0
:1012E00074656E6E6120526F746F7220436F6E74FE
:1012F000726F6C6C657220762E20000056657273DA
:10130000696F6E2000005061726B696E6720415AF0
:101310003D00417A696D757468206F666673657407
:101320003D200000417A696D757468206F666673B0
:1013300065742073617665640000456C6576617440
:10134000696F6E206F66667365743D200000456CA2
:1013500065766174696F6E206F666673657420735D
:101360006176656400002D2D2D2D2D2D2D2D2D2D1B
:101370002D2D2D2D434F4D4D414E44204C4953545E
:101380002D2D2D2D2D2D2D2D2D2D2D2D2D2D0000E7
:101390003F202048656C702054657874000041201F
:1013A0002043572F43435720526F746174696F6E07
:1013B0002053746F7000422020416E74656E6E6120
:1013C00020446972656374696F6E20454C00432048
:1013D00020416E74656E6E61204469726563746944
:1013E0006F6E20415A00433220416E74656E6E610B
:1013F00020446972656374696F6E20415A26454CBA
:101400000000442020446F776E2044697265637445
:10141000696F6E20526F746174696F6E00004520B1
:101420002055502F444F574E2044697265637469AC
:101430006F6E20526F746174696F6E2053746F7099
:101440000000462020536574206D6178696D616CE1
:1014500020706F736974696F6E20696E20617A699C
:101460006D7574683A204661616100004621205321
:101470006176652063757272656E7420706F736932
:1014800074696F6E206173206D6178696D616C2085
:10149000706F736974696F6E0000463F2053686F08
:1014A00077206D6178696D616C20706F7369746904
:1014B0006F6E20696E20617A696D757468004720CF
:1014C00020536574204F666673657420496E20450D
:1014D0004C3A204765656500473F2053686F772089
:1014E0004F666673657420436F6E7374616E74200B
:1014F000666F7220454C000048202048656C7020C3
:1015000074657874000049202053686F77207061FB
:1015100072616D657465727300004A44205365748E
:1015200020426565706572206F6E202D20446972BF
:101530006563742043757272656E74004A46205369
:10154000657420426565706572206F6E202D20469F
:1015500072657175656E637900004A4E205365743B
:1015600020426565706572206F6666004A6E205382
:101570006574206265657065722066726571756557
:101580006E637920286E203D20313030302D31308F
:1015900030303020487A29004B2020416E74656E2F
:1015A0006E6120446972656374696F6E205365745F
:1015B00074696E6720496E20454C3A204B6565651D
:1015C00000004C2020436F756E74657220436C6F71
:1015D000636B7769736520286C6566742920526F88
:1015E000746174696F6E00004D2020416E74656EE9
:1015F0006E6120446972656374696F6E205365740F
:1016000074696E6720496E20415A3A204D616161CC
:1016100000004E202054797065206F662064697345
:10162000706C617900004F20204F666673657420EE
:10163000496E20415A004F3F2053686F77204F6614
:101640006673657420436F6E7374616E74004F210E
:1016500020536176652063757272656E7420706FB9
:10166000736974696F6E2061732053544F502070FA
:101670006F736974696F6E005020205061726B69DE
:101680006E6720546F3A2050616161206565650086
:10169000502120536176652063757272656E7420E7
:1016A000706F736974696F6E206173207061726B03
:1016B000696E672076616C7565730000503F20533A
:1016C000686F77207361766564207061726B696EF4
:1016D000672076616C75657300005120205072653B
:1016E000636973696F6E20302E31202D20302E35C6
:1016F000202D20312E3020646567000052202043C9
:101700006C6F636B776973652028726967687429E9
:1017100020526F746174696F6E00532020416C6CAD
:101720002053746F7000546E20436F6D2E20706FC5
:10173000727420737065656420286E3D34383030D3
:101740002C393630302C31393230302C333834307B
:10175000302C353736303029000055202055702088
:10176000446972656374696F6E20526F7461746945
:101770006F6E0000562020536F667476617265208C
:1017800056657273696F6E00572020416E74656EE6
:101790006E6120446972656374696F6E205365746D
:1017A00074696E673A205761616120656565000064
:1017B0005920204543484F204F4E202F204F46466A
:1017C00000005A2020537769746368207A65726F2D
:1017D00020706F736974696F6E20746F204E6F7222
:1017E00064202F20536F7574680026202053657481
:1017F000206D6178696D756D20656C6576617469C1
:101800006F6E2028313830202D20666C6970206F73
:101810006E3B203930202D20666C6970206F666623
:101820002900252020456C65766174696F6E206300
:101830006F6E74726F6C204F4E202F204F46460003
:101840002A20204D61782E20656C65766174696F61
:101850006E20666F72206F7665727475726E696E37
:101860006700232020456D756C6174696F6E206F71
:101870006620475332333241202F204753323332D0
:1018800042003C2020417A696D7574682063616C68
:101890006962726174696F6E00005E2020456C653C
:1018A000766174696F6E2063616C696272617469DC
:1018B0006F6E00005B20204F776E20636F6F726445
:1018C000696E617465202D206C617469747564653E
:1018D00000005D20204F776E20636F6F7264696E29
:1018E000617465202D206C6F6E6769747564650086
:1018F00061616120497320416E2056616C756520DD
:10190000466F722054686520417A696D757468204D
:1019100028302D3336302900656565204973204114
:101920006E2056616C756520466F72205468652084
:10193000456C65766174696F6E2028302D313830C2
:101940002900446973706C61792074797065200096
:10195000302E3500302E3100312E3000302E320046
:10196000507265636973696F6E2073657420746F5C
:1019700020005A65726F20706F736974696F6E20F2
:101980006F6E20004D6178696D756D20656C6576B0
:101990006174696F6E2069732000426565706572BD
:1019A00000003A204672657175656E6379003A20D1
:1019B0004469726563742063757272656E740000A9
:1019C000206672657175656E63793A200000434F39
:1019D0004D20706F72742073706565643A2000004A
:1019E0005468652073706565642077696C6C206F3E
:1019F0006E6C792062652076616C69642061667422
:101A00006572207265626F6F7400434F4D20737072
:101A1000656564206973206E6F74207265636F6DF5
:101A20006D656E6465642E20596F752062657474EF
:101A300065722075736520343830302C393630307B
:101A40002C31393230302C33383430302C35373675
:101A5000303000005265626F6F74206E6F773F20E8
:101A60002879203D20796573206F74686572203D68
:101A7000206E6F2900004E657720434F4D20737014
:101A80006565642061637469766174656400456CA2
:101A900065766174696F6E20697320004D617869A5
:101AA0006D756D206F6620617A696D7574683D2073
:101AB000000056616C756520736176656400547929
:101AC00070653A204753323332002D2D2D2D2D2DA8
:101AD0002D4C495354204F4620504152414D4554BE
:101AE0004552532D2D2D2D2D2D2D00004F66667343
:101AF0006574206F6620617A696D7574683A20009C
:101B00004F6666736574206F6620656C65766174D8
:101B1000696F6E3A20004D6178696D756D20706F48
:101B2000736974696F6E206F6620617A696D757470
:101B3000683A20004D6178696D756D20706F73692A
:101B400074696F6E206F6620656C65766174696F6D
:101B50006E3A20004D61782E20656C65766174695F
:101B60006F6E20666F72206F7665727475726E6923
:101B70006E673A200000456C65766174696F6E206F
:101B8000636F6E74726F6C3A20005061726B696E95
:101B900067206F6E20415A3A20005A65726F20709C
:101BA0006F736974696F6E3A2000434F4D20706FF8
:101BB0007274206563686F3A2000426565706572D3
:101BC0003A2000004672657175656E63790044695C
:101BD000726563742043757272656E7400004265AD
:101BE00065706572206672657175656E63793A20FD
:101BF0000000507265636973696F6E3A2000446932
:101C000073706C617920747970653A2000004C61C2
:101C10007469747564653A20000020204C6F6E670B
:101C200069747564653A2000536F667477617265F4
:101C30002076657273696F6E3A20000046455252F5
:101C40003A200000204F4552523A20004172652050
:101C5000796F7520737572653F00417A696D75748F
:101C6000682069732063616C6962726174656400E5
:101C7000417A696D7574682063616C696272617420
:101C8000696E67206572726F7200456C657661746B
:101C9000696F6E2069732063616C6962726174653B
:101CA0006400456C65766174696F6E2063616C6970
:101CB00062726174696E67206572726F72006C6126
:101CC0007469747564653A2000006C6F6E6769749E
:101CD0007564653A2000454C3A204572726F720077
:101CE000415A3A204572726F7200444F574E205548
:101CF000502053544F502043435720204357000057
:101D0000415A494D5554483A2000415A494D55547D
:101D1000483A204572726F72202020202020000057
:101D2000202020202020202053544F502043435770
:101D300020204357000020202020202020204D4537
:101D40004E55202020202020202000002020202070
:101D50002020202020202020202020202020202083
:101D6000000053455420415A494D55544820544F82
:101D70002020000053455420454C455641542E2008
:101D8000544F202000005041524B494E4720415AA9
:101D9000494D5554482000005041524B2E20454C8F
:101DA00045564154494F4E200000415A494D555423
:101DB00048204F464653455420200000454C455688
:101DC00041542E204F4646534554202000004D419B
:101DD00058494D554D20415A494D55544820000011
:101DE0004D415820454C202D204F564552542E2011
:101DF000000054595045204F4620444953504C410F
:101E00005920200020204C454420204C4344000011
:101E1000454C45564154494F4E20434F4E54522E47
:101E20002000434F4D4D554E49434154494F4E209C
:101E300047533233320020202041202020204220EE
:101E400000004D4158494D554D20454C4556415493
:101E50002E20000020202039302020313830000092
:101E60005A45524F20504F494E54204F4E200000AB
:101E70004E4F524420200000534F5554482000003C
:101E8000202020204E202020532000004245455095
:101E90004552202020004F46462020202020202090
:101EA0002000446972656374204375722E004652A7
:101EB000455155454E435920200020204F4646208D
:101EC000204443202046525100004652455155457A
:101ED0004E43593A2020000020202020566572737E
:101EE000696F6E200000505245434953494F4E20C0
:101EF0002000302E3120646567202000302E3220F3
:101F0000646567202000302E35206465672020003E
:101F1000312E302064656720200053455420415302
:101F20004C20544F202020004155544F20545552EE
:101F30004E494E472020202020004F5645525455F0
:101F4000524E494E4720202020202000434F4D2054
:101F5000535045454420202020202000434F4D2051
:101F6000504F5254204543484F20495320004E4D76
:101F7000454120544553542020202020202020007B
:101F800043414C4942524154494F4E2020415A4905
:101F900020454C450000202020415A4920454C4511
:101FA000000043414C4942524154494F4E20504C4D
:101FB0005320574149540000202020202020202079
:101FC0000000202020202020200047474100202022
:101FD000204F464620204F4E00004C6174697475B6
:101FE00064653A20202000004C6F6E676974756448
:101FF000653A20002020204F4B2020200000303167
:10200000323334353637383941424344454630312E
:102010003233343536373839414243444546400E31
:102020003E6E006ACF0EAF6EB06A240EAC6E900E9C
:10203000AB6E000124EE47F00F0EC16E070EB46EBA
:1020400003018E6B8D6B080E8C6F830E8B6F0001FE
:10205000896A8A6A8B6A8C6A8D6AC00E926E870E54
:10206000936EBE0E946ED00E956E880E966E310EE7
:10207000CD6EB16A250E9D6EA06A0B0EBD6EFA0E76
:10208000BF6EBE6ABA6AF40ED36E400E9B6EC00E6F
:10209000F26E700EF16E900EF06E9F8A9F94D08E4D
:1020A000F188F088070EB46EC66AC26A0F0EC16E60
:1020B000C06A900EAB6E200EAC6E080EB86EAC9877
:1020C000AC84030EB06E400EAF6E02EE12F0120E34
:1020D000F76EA00EF66E1FEC03F0EF6A0301020E1E
:1020E000566F200E886F93988A9893968A96939A43
:1020F0008A9A939C8A9C95968C9695928C929590B0
:102100008C9094908B90429E4390516B526B506B8D
:10211000449C429C439E336B326B316B306B376B0C
:10212000366B356B346B448281A04492448481A227
:102130004494448844860001AA6BBD6BBC6BBF6BA2
:10214000BE6B0301640E5B6F0001A76BA86B010EF1
:10215000966F810EDA6FED0EDB6F430EDC6F490E6A
:10216000DD6F2D0EDE6F190EDF6F110EE06FCD0EDD
:10217000E16F010EE26F090EE36FE469170EE56F80
:10218000930EE66F310EE76F750EE86F070EE96F7D
:10219000130EEA6F850EEB6FF10EEC6F050EED6F0F
:1021A000B30EEE6F910EEF6F710EF06F770EF16F51
:1021B000330EF26FF70EF36F7F0EF46F610EF56F53
:1021C000640E14EC02F0FE0E43EC01F0400E43EC02
:1021D00001F0000E43EC01F0040E43EC01F0040E9C
:1021E00043EC01F0040E43EC01F0150E43EC01F05A
:1021F0000E0E43EC01F0040E43EC01F0000E43EC34
:1022000001F01E0E14EC02F0FE0E43EC01F0480E3D
:1022100043EC01F0000E43EC01F0040E43EC01F03E
:102220000E0E43EC01F0150E43EC01F0040E43ECEE
:1022300001F0040E43EC01F0040E43EC01F0000E3B
:1022400043EC01F01E0E14EC02F0FE0E43EC01F024
:10225000500E43EC01F0000E43EC01F0040E43EC91
:1022600001F0020E43EC01F01F0E43EC01F0020EF0
:1022700043EC01F0040E43EC01F0000E43EC01F0DE
:10228000000E43EC01F01E0E14EC02F0FE0E43ECC7
:1022900001F0580E43EC01F0000E43EC01F0040E87
:1022A00043EC01F0080E43EC01F01F0E43EC01F08B
:1022B000080E43EC01F0040E43EC01F0000E43EC79
:1022C00001F0000E43EC01F01E0E14EC02F0FE0EC5
:1022D00043EC01F0600E43EC01F0000E43EC01F022
:1022E000010E43EC01F0050E43EC01F0090E43EC46
:1022F00001F01F0E43EC01F0080E43EC01F0040E58
:1023000043EC01F0000E43EC01F01E0E14EC02F061
:10231000FE0E43EC01F0680E43EC01F0040E43ECBA
:1023200001F00A0E43EC01F0040E43EC01F0000E44
:1023300043EC01F0000E43EC01F0000E43EC01F021
:10234000000E43EC01F0000E43EC01F01E0E14EC05
:1023500002F0AA6A210EA96EE4EC01F00301896F74
:10236000E4EC01F003018A6FAA6AA96AE4EC01F0C7
:102370004A6EE4EC01F04B6EAA6A020EA96EE4EC20
:1023800001F04C6EE4EC01F04D6EAA6A040EA96EE9
:10239000E4EC01F0676EE4EC01F0686EAA6A060EE8
:1023A000A96EE4EC01F0696EE4EC01F06A6EAA6AD1
:1023B000080EA96EE4EC01F06F6EE4EC01F0706EB3
:1023C000AA6A0A0EA96EE4EC01F0716EE4EC01F069
:1023D000726EAA6A0C0EA96EE4EC01F0736EE4EC66
:1023E00001F0746EAA6A0E0EA96EE4EC01F0666E3E
:1023F000AA6A0F0EA96EE4EC01F000019A6FAA6AB6
:102400001E0EA96EE4EC01F09B6FAA6A100EA96E75
:10241000E4EC01F00301596FAA6A110EA96EE4EC15
:1024200001F00301556FAA6A1F0EA96EE4EC01F0DA
:102430000001B86FE4EC01F0B96FAA6A120EA96E40
:10244000E4EC01F003013A6FE4EC01F003013B6FAF
:10245000E4EC01F003013C6FE4EC01F003013D6F9B
:10246000AA6A160EA96EE4EC01F003013E6FE4ECDB
:1024700001F003013F6FE4EC01F00301406FE4EC75
:1024800001F00301416FAA6A1A0EA96EE4EC01F093
:102490000301426FE4EC01F00301436FAA6A1C0ED2
:1024A000A96EE4EC01F00301856FE4EC01F0030197
:1024B000866F86510A0DF3CF86F385510A0DF3CF4F
:1024C00085F3F4508627166A070E156EA10E146E5A
:1024D000200E136E85C31BF086C31CF01D6A1E6A96
:1024E00036EC02F014C084F313C083F3020E030130
:1024F000555DD8A4010E3B6E040E555DD8A4010EA7
:102500003B160A0E555DD8A4010E3B16140E555D00
:10251000D8A4010E3B16000103E00301040E556F21
:10252000000194EC43F09B311CE30EEC00F0120E22
:10253000F76EB60EF66E3BEC01F0120EF76ECC0E97
:10254000F66E3BEC01F0800E016E8EC329F08DC358
:1025500028F08CC327F08BC326F0010EA7EC00F007
:1025600026D0840E026E020E086E840E036E010EDB
:10257000046E050E096EED51136EEBEC01F0E8519F
:10258000136EEBEC01F0F251136EEBEC01F0E6513F
:10259000136EEBEC01F0F051136EEBEC01F0E8512F
:1025A000136EEBEC01F096948D8496948D94120E3C
:1025B000F76EDE0EF66EAFEC01F0040E016E8EC308
:1025C00029F08DC328F08CC327F08BC326F0010EB1
:1025D000A7EC00F00D0EB7EC01F00A0EB7EC01F01D
:1025E0004BC057F04AC056F04DC059F04CC058F09F
:1025F00003015551B40DF3CFC4F0F4CFC5F05551DC
:10260000680DF3CFC6F0F4CFC7F00001C7276650BE
:1026100003015503F4CFC9F0F3CFC8F055510A0DAB
:10262000F3CFCAF0F4CFCBF05551640DF3CFCCF01B
:10263000F4CFCDF055511E0DF3CFD0F0F4CFD1F043
:102640005551320DF3CFCEF0F4CFCFF055510F0DE1
:10265000F3CFD2F0F4CFD3F042944296429042921C
:102660004DC049F04CC048F000019A51E8BA01D081
:10267000938E070E186ED00E15EC02F001EE47F0A7
:10268000EF6A00EEF6F0EF6A449C6AEC40F0ABA211
:1026900005D0AB98AB880301894B8A2B0001ABA412
:1026A00004D0AECFA9F003018A2B0001010E42B481
:1026B000000E3B6E010E42B0000E3B16D8B454D053
:1026C00082B428D081A604D093968A96E7EC43F092
:1026D0004590458293988A8882B41CD06AEC40F079
:1026E00088EC26F04A50565C136E4B505758146EC7
:1026F00003EC03F00B6E14C00CF0D2510B5CD35101
:102700000C580C50D319D8B0800A03E74284959630
:102710008C86E2D782B628D081A804D093988A9874
:10272000E7EC43F04580459293968A8682B61CD0AA
:102730006AEC40F088EC26F04A50565C136E4B5021
:102740005758146E03EC03F00B6E14C00CF0D2510A
:102750000B5CD3510C580C50D319D8B0800A03E746
:10276000428495968C86E2D7000E42B4010E3B6EF1
:10277000000E42B0010E3B1227E0010E82B4000EA3
:102780003B6E010E82B6000E3B12010E82B2000EAD
:102790003B1219E093968A9693988A9842944290B5
:1027A000449C010E82B4000E3B6E010E82B6000EF8
:1027B0003B12010E82B2000E3B1205E06AEC40F0C3
:1027C00088EC26F0EED704D093968A9693988A9850
:1027D0009A51E8B27FD0010E42B6000E3B6E010E58
:1027E00042B2000E3B16D8B454D080BC28D081AC85
:1027F00004D0939C8A9CE7EC43F045964584939AD9
:102800008A8A80BC1CD06AEC40F088EC26F04C50E0
:10281000585C136E4D505958146E03EC03F00B6E58
:1028200014C00CF0CA510B5CCB510C580C50CB1996
:10283000D8B0800A03E7428695968C86E2D780BEA0
:1028400028D081AA04D0939A8A9AE7EC43F045866F
:102850004594939C8A8C80BE1CD06AEC40F088EC36
:1028600026F04C50585C136E4D505958146E03ECC2
:1028700003F00B6E14C00CF0CA510B5CCB510C581A
:102880000C50CB19D8B0800A03E7428695968C8607
:10289000E2D7000E42B6010E3B6E000E42B2010EB0
:1028A0003B1214E0010E80BC000E3B6E010E80BE98
:1028B000000E3B12010E82B2000E3B1206E0939C0A
:1028C0008A9C939A8A9A4296429204D0939C8A9CBC
:1028D000939A8A9A6F504A5C4E6E70504B584F6E66
:1028E00071504C5C506E72504D58516E42A426D0BF
:1028F000000E45B0010E3B6EC6514E5CC7514F589D
:102900004F50C719D8B0800A02E6000E01D0010E60
:102910003B1603E093968A964294000E45B2010E50
:102920003B6E4FBE05D04E504F1002E0000E01D05E
:10293000010E3B1603E093988A98429442A626D053
:10294000000E45B4010E3B6EC851505CC951515840
:102950005150C919D8B0800A02E6000E01D0010E0C
:102960003B1603E0939A8A9A4296000E45B6010EF2
:102970003B6E51BE05D05050511002E0000E01D008
:10298000010E3B1603E0939C8A9C429682A276EC51
:102990002CF0000E42B4010E3B6E000E42B6010E4A
:1029A0003B1201E0449C010E42B4000E3B6E010E4E
:1029B00042B6000E3B16010E42B0000E3B16010E51
:1029C00042B2000E3B1602E095968C9642BC828085
:1029D00042AC829088EC26F0000E80BE010E3B6E69
:1029E000000E80BC010E3B1604E04DC059F04CC0F7
:1029F00058F0000E82B4010E3B6E000E82B6010E3E
:102A00003B1604E04BC057F04AC056F0000E44BCE1
:102A1000010E3B6E000E42BC010E3B1618E0AB539C
:102A200016E0146AABC013F0186A460E176E61EC1C
:102A300002F01CC00CF01BC00BF00C500B1002E19C
:102A400026EC40F0AB07010E14EC02F0E8D7000EC4
:102A500044BC010E3B6E010E82B0000E3B16D8B492
:102A600067EF25F0449CF651B16F240EB15D04E18F
:102A700081EC38F063EF25F0570EB15DD8A47BD020
:102A8000FA510B6E200E0B5CD8A473D001EE98F0B7
:102A900010EEF6F0060EF36E030E2EEC03F0EF6A66
:102AA00004EE15F011EE98F0060E27EC03F0A2EC00
:102AB0004AF0AEC3B3F0ADC3B2F0B351E8AE02D04A
:102AC000000E01D0010E3B6EB351E8BE07D0B353E8
:102AD00003E1B251B40802E2000E01D0010E3B1630
:102AE0000001D8B444D0B3C094F3B2C093F334EC33
:102AF00044F096C349F095C348F001EE98F010EE0B
:102B0000F6F0020EF36E030E2EEC03F0EF6A04EE05
:102B100015F011EE98F0060E27EC03F0A2EC4AF047
:102B2000AEC3B3F0ADC3B2F0B351E8AE02D0000E05
:102B300001D0010E3B6EB351E8BE09D0010EB35D6A
:102B400006E303E1690EB25D02E3000E01D0010E5F
:102B50003B1600010CE0B3C090F3B2C08FF3F8EC69
:102B600043F092C347F091C346F026EC40F0429404
:102B7000429663EF25F04D0EB15DD8A488D0F75191
:102B80000B6E520E0B5C0FE126EC40F081A804D0D6
:102B900093988A98E7EC43F04580459293968A860D
:102BA0004284429072D04C0E0B5C0FE126EC40F058
:102BB00081A604D093968A96E7EC43F0459045822F
:102BC00093988A884284429060D0550E0B5C0FE146
:102BD00026EC40F081AC04D0939C8A9CE7EC43F057
:102BE00045964584939A8A8A428642924ED0440EF4
:102BF0000B5C0FE126EC40F081AA04D0939A8A9AEC
:102C0000E7EC43F045864594939C8A8C4286429239
:102C10003CD001EE98F010EEF6F0020EF36E030ECB
:102C20002EEC03F0EF6A04EE15F011EE98F0060EAC
:102C300027EC03F0A2EC4AF0AEC3B3F0ADC3B2F0A0
:102C4000B351E8AE02D0000E01D0010E3B6EB3517D
:102C5000E8BE09D0010EB35D06E303E1690EB25D83
:102C600002E3000E01D0010E3B1600010EE0B3C0DE
:102C700090F3B2C08FF3F8EC43F092C347F091C3E6
:102C800046F026EC40F04280429463EF25F04B0E74
:102C9000B15D3CE101EE98F010EEF6F0020EF36E3D
:102CA000030E2EEC03F0EF6A04EE15F011EE98F02F
:102CB000060E27EC03F0A2EC4AF0AEC3B3F0ADC3AE
:102CC000B2F0B351E8AE02D0000E01D0010E3B6E5F
:102CD000B351E8BE07D0B35303E1B251B40802E2E6
:102CE000000E01D0010E3B1600010EE0B3C094F3BC
:102CF000B2C093F334EC44F096C349F095C348F066
:102D000026EC40F04282429663EF25F0520EB15D10
:102D100010E126EC40F081A804D093988A98E7EC63
:102D200043F04580459293968A864284429063EFB1
:102D300025F04C0EB15D10E126EC40F081A604D0E8
:102D400093968A96E7EC43F04590458293988A885B
:102D50004284429063EF25F0550EB15D10E126EC00
:102D600040F081AC04D0939C8A9CE7EC43F04596FC
:102D70004584939A8A8A4286429263EF25F0440EF4
:102D8000B15D10E126EC40F081AA04D0939A8A9AB2
:102D9000E7EC43F045864594939C8A8C42864292A8
:102DA00063EF25F0530EB15D24E1F7510B6E410E38
:102DB0000B5C07E193968A9693988A984290429486
:102DC00016D0450E0B5C07E1939A8A9A939C8A9CD5
:102DD000429242960CD093968A9693988A98939AA8
:102DE0008A9A939C8A9C429042924294429663EFC4
:102DF00025F0410EB15DD8A49AD0F7510B6E5A0E52
:102E00000B5CD8A48CD001EE98F010EEF6F0030E17
:102E1000F36E2EEC03F0EF6A04EE15F011EE98F06D
:102E2000060E27EC03F0A2EC4AF0AEC3B3F0ADC33C
:102E3000B2F0B351E8AE02D0000E01D0010E3B6EED
:102E4000B351E8BE09D0010EB35D06E303E1690E9C
:102E5000B25D02E3000E01D0010E3B160001D8B4B2
:102E60005DD0B3C090F3B2C08FF3F8EC43F092C3DF
:102E700047F091C346F0FD510B6E200E0B5C010E26
:102E8000D8A4000E3B6EFE510B6E450E0B5C010E7E
:102E9000D8A4000E3B16FF510B6E4C0E0B5C010EBE
:102EA000D8A4000E3B1636E001EE98F010EEF6F0D6
:102EB0000B0EF36E030E2EEC03F0EF6A04EE15F02A
:102EC00011EE98F0060E27EC03F0A2EC4AF0AEC328
:102ED000B3F0ADC3B2F0B351E8AE02D0000E01D0F2
:102EE000010E3B6EB351E8BE07D0B35303E1B251BC
:102EF000B40802E2000E01D0010E3B1600010AE008
:102F0000B3C094F3B2C093F334EC44F096C349F0E9
:102F100095C348F04294429626EC40F006D0939632
:102F20008A9693988A984290429463EF25F0450ED2
:102F3000B15DD8A447D0F7510B6E4C0E0B5C3AE153
:102F400001EE98F010EEF6F0030EF36E2EEC03F0A7
:102F5000EF6A04EE15F011EE98F0060E27EC03F080
:102F6000A2EC4AF0AEC3B3F0ADC3B2F0B351E8AED9
:102F700002D0000E01D0010E3B6EB351E8BE07D067
:102F8000B35303E1B251B40802E2000E01D0010EC6
:102F90003B1600010EE0B3C094F3B2C093F334ECDF
:102FA00044F096C349F095C348F04282429626EC1D
:102FB00040F006D0939A8A9A939C8A9C42924296B9
:102FC00063EF25F0430EB15DD8A4BED0F7510B6E70
:102FD000320E0B5CD8A473D09A51E8B435D02B0EC6
:102FE000B7EC01F0300EB7EC01F0040E016E030EE9
:102FF000076E4FC022F04EC021F055C31BF01C6A73
:1030000078EC02F01B6E14C01CF06FEC00F02B0E7D
:10301000B7EC01F0300EB7EC01F0030E076E51C0B3
:1030200022F050C021F055C31BF01C6A78EC02F06E
:103030001B6E14C01CF06FEC00F00D0EB7EC01F02D
:103040000A0EB7EC01F03AD0410EB7EC01F05A0E7F
:10305000B7EC01F03D0EB7EC01F0040E016E030E6B
:10306000076E4FC022F04EC021F055C31BF01C6A02
:1030700078EC02F01B6E14C01CF06FEC00F0450EF3
:10308000B7EC01F04C0EB7EC01F03D0EB7EC01F0DF
:10309000030E076E51C022F050C021F055C31BF043
:1030A0001C6A78EC02F01B6E14C01CF06FEC00F090
:1030B0000D0EB7EC01F00A0EB7EC01F043D09A51B7
:1030C000E8B41FD02B0EB7EC01F0300EB7EC01F0D6
:1030D000040E016E030E076E4FC022F04EC021F0A9
:1030E00055C31BF01C6A78EC02F01B6E14C01CF078
:1030F0006FEC00F00D0EB7EC01F00A0EB7EC01F02A
:1031000021D0410EB7EC01F05A0EB7EC01F03D0EA4
:10311000B7EC01F0040E016E030E076E4FC022F0F3
:103120004EC021F055C31BF01C6A78EC02F01B6EF8
:1031300014C01CF06FEC00F00D0EB7EC01F00A0E9D
:10314000B7EC01F063EF25F0420EB15D45E19A5115
:10315000E8B41FD02B0EB7EC01F0300EB7EC01F045
:10316000040E016E030E076E51C022F050C021F014
:1031700055C31BF01C6A78EC02F01B6E14C01CF0E7
:103180006FEC00F00D0EB7EC01F00A0EB7EC01F099
:1031900021D0450EB7EC01F04C0EB7EC01F03D0E1E
:1031A000B7EC01F0040E016E030E076E51C022F061
:1031B00050C021F055C31BF01C6A78EC02F01B6E66
:1031C00014C01CF06FEC00F00D0EB7EC01F00A0E0D
:1031D000B7EC01F063EF25F0560EB15D3AE1F7511F
:1031E0000B6E450E0B5C1AE1560EB7EC01F0450E66
:1031F000B7EC01F0040E016E8EC329F08DC328F0E8
:103200008CC327F08BC326F0010EA7EC00F00D0E47
:10321000B7EC01F00A0EB7EC01F019D0120EF76E00
:10322000FC0EF66EAFEC01F0040E016E8EC329F0B9
:103230008DC328F08CC327F08BC326F0010EA7ECBA
:1032400000F00D0EB7EC01F00A0EB7EC01F063EFE1
:1032500025F0500EB15DD8A4FFD0F7510B6E3F0E94
:103260000B5C3BE1130EF76E060EF66EAFEC01F051
:10327000040E016E030E076E68C022F067C021F0D5
:1032800055C31BF01C6A78EC02F01B6E14C01CF0D6
:103290006FEC00F0200EB7EC01F0450EB7EC01F03A
:1032A0004C0EB7EC01F03D0EB7EC01F0030E076ECB
:1032B0006AC022F069C021F055C31BF01C6A78EC8B
:1032C00002F01B6E14C01CF06FEC00F00D0EB7EC9A
:1032D00001F00A0EB7EC01F0BDD0F7510B6E210ED4
:1032E0000B5C1BE14BC068F04AC067F04DC06AF050
:1032F0004CC069F0AA6A040EA96E6750CFEC01F0C9
:103300006850CFEC01F0AA6A060EA96E6950CFECA6
:1033100001F06A50CFEC01F09DD0F7510301BD6F71
:10332000000171EC4BF045AE89D001EE98F010EE43
:10333000F6F0020EF36E030E2EEC03F0EF6A04EECD
:1033400015F011EE98F0060E27EC03F0A2EC4AF00F
:10335000AEC3B3F0ADC3B2F0B351E8BE09D0010EB5
:10336000B35D06E303E1690EB25D02E3000E01D036
:10337000010E3B6E0001B351E8AE02D0000E01D049
:10338000010E3B1612E0B25103015503F3CF67F073
:10339000F4CF68F00001B35103015503F3506826E0
:1033A00055AF03D00001B251685E000101EE98F004
:1033B00010EEF6F0060EF36E030E2EEC03F0EF6A3D
:1033C00004EE15F011EE98F0060E27EC03F0A2ECD7
:1033D0004AF0AEC3B3F0ADC3B2F0B351E8BE2DD0E6
:1033E000B3BF05D0B35116E1B50EB25D13E20001D3
:1033F000B25103015503F3CF69F0F4CF6AF0000135
:10340000B35103015503F3506A2655AF03D00001B1
:10341000B2516A5E0001AA6A040EA96E6750CFEC31
:1034200001F06850CFEC01F0AA6A060EA96E69504F
:10343000CFEC01F06A50CFEC01F00CD068C047F03F
:1034400067C046F06AC049F069C048F042804282D5
:103450004294429663EF25F04F0EB15DD8A494D00C
:10346000F7510B6E3F0E0B5C1EE1130EF76E120E42
:10347000F66EAFEC01F0040E016E076A70C022F028
:103480006FC021F055C31BF01C6A78EC02F01B6E74
:1034900014C01CF06FEC00F00D0EB7EC01F00A0E3A
:1034A000B7EC01F06FD0F7510B6E210E0B5C16E1FB
:1034B000AA6A080EA96E4A50CFEC01F04B50CFEC2F
:1034C00001F0130EF76E240EF66EAFEC01F00D0E48
:1034D000B7EC01F00A0EB7EC01F054D001EE98F011
:1034E00010EEF6F0020EF36E030E2EEC03F0EF6A10
:1034F00004EE15F011EE98F0060E27EC03F0A2ECA6
:103500004AF0AEC3B3F0ADC3B2F0B351E8AE02D0EF
:10351000000E01D0010E3B6EB351E8BE07D0B3538D
:1035200003E1B251320802E2000E01D0010E3B1657
:10353000000127E0B25103015503F3CF6FF0F4CF40
:1035400070F00001B35103015503F350702655AFDD
:1035500003D00001B251705EAA6A080EA96E6F50C6
:10356000CFEC01F07050CFEC01F0130EF76E240E8B
:10357000F66EAFEC01F00D0EB7EC01F00A0EB7ECF1
:1035800001F0000163EF25F0470EB15DD8A479D0BA
:10359000F7510B6E3F0E0B5C1EE1130EF76E3A0EE9
:1035A000F66EAFEC01F0040E016E076A72C022F0F5
:1035B00071C021F055C31BF01C6A78EC02F01B6E41
:1035C00014C01CF06FEC00F00D0EB7EC01F00A0E09
:1035D000B7EC01F054D001EE98F010EEF6F0020EC8
:1035E000F36E030E2EEC03F0EF6A04EE15F011EE0D
:1035F00098F0060E27EC03F0A2EC4AF0AEC3B3F04D
:10360000ADC3B2F0B351E8AE02D0000E01D0010E4E
:103610003B6EB351E8BE07D0B35303E1B2511E086D
:1036200002E2000E01D0010E3B16000127E0B2516C
:1036300003015503F3CF71F0F4CF72F00001B351E1
:1036400003015503F350722655AF03D00001B25168
:10365000725EAA6A0A0EA96E7150CFEC01F0725028
:10366000CFEC01F0130EF76E4E0EF66EAFEC01F0DC
:103670000D0EB7EC01F00A0EB7EC01F0000163EF9C
:1036800025F0480EB15D04E03F0EB15DD8A442D2F2
:10369000130EF76E660EF66EAFEC01F00D0EB7EC82
:1036A00001F00A0EB7EC01F0130EF76E900EF66EF5
:1036B000AFEC01F00D0EB7EC01F00A0EB7EC01F023
:1036C000130EF76E9E0EF66EAFEC01F00D0EB7EC1A
:1036D00001F00A0EB7EC01F0130EF76EB60EF66E9F
:1036E000AFEC01F00D0EB7EC01F00A0EB7EC01F0F3
:1036F000130EF76ECE0EF66EAFEC01F00D0EB7ECBA
:1037000001F00A0EB7EC01F0130EF76EE60EF66E3E
:10371000AFEC01F00D0EB7EC01F00A0EB7EC01F0C2
:10372000140EF76E020EF66EAFEC01F00D0EB7EC54
:1037300001F00A0EB7EC01F0140EF76E1E0EF66ED5
:10374000AFEC01F00D0EB7EC01F00A0EB7EC01F092
:10375000140EF76E420EF66EAFEC01F00D0EB7ECE4
:1037600001F00A0EB7EC01F0140EF76E6C0EF66E57
:10377000AFEC01F00D0EB7EC01F00A0EB7EC01F062
:10378000140EF76E9A0EF66EAFEC01F00D0EB7EC5C
:1037900001F00A0EB7EC01F0140EF76EBE0EF66ED5
:1037A000AFEC01F00D0EB7EC01F00A0EB7EC01F032
:1037B000140EF76ED80EF66EAFEC01F00D0EB7ECEE
:1037C00001F00A0EB7EC01F0140EF76EF80EF66E6B
:1037D000AFEC01F00D0EB7EC01F00A0EB7EC01F002
:1037E000150EF76E060EF66EAFEC01F00D0EB7EC8F
:1037F00001F00A0EB7EC01F0150EF76E1A0EF66E18
:10380000AFEC01F00D0EB7EC01F00A0EB7EC01F0D1
:10381000150EF76E3C0EF66EAFEC01F00D0EB7EC28
:1038200001F00A0EB7EC01F0150EF76E5A0EF66EA7
:10383000AFEC01F00D0EB7EC01F00A0EB7EC01F0A1
:10384000150EF76E6C0EF66EAFEC01F00D0EB7ECC8
:1038500001F00A0EB7EC01F0150EF76E980EF66E39
:10386000AFEC01F00D0EB7EC01F00A0EB7EC01F071
:10387000150EF76EC20EF66EAFEC01F00D0EB7EC42
:1038800001F00A0EB7EC01F0150EF76EE80EF66EB9
:10389000AFEC01F00D0EB7EC01F00A0EB7EC01F041
:1038A000160EF76E120EF66EAFEC01F00D0EB7ECC1
:1038B00001F00A0EB7EC01F0160EF76E260EF66E4A
:1038C000AFEC01F00D0EB7EC01F00A0EB7EC01F011
:1038D000160EF76E360EF66EAFEC01F00D0EB7EC6D
:1038E00001F00A0EB7EC01F0160EF76E4E0EF66EF2
:1038F000AFEC01F00D0EB7EC01F00A0EB7EC01F0E1
:10390000160EF76E780EF66EAFEC01F00D0EB7ECFA
:1039100001F00A0EB7EC01F0160EF76E900EF66E7F
:10392000AFEC01F00D0EB7EC01F00A0EB7EC01F0B0
:10393000160EF76EBC0EF66EAFEC01F00D0EB7EC86
:1039400001F00A0EB7EC01F0160EF76EDA0EF66E05
:10395000AFEC01F00D0EB7EC01F00A0EB7EC01F080
:10396000160EF76EFC0EF66EAFEC01F00D0EB7EC16
:1039700001F00A0EB7EC01F0170EF76E1A0EF66E94
:10398000AFEC01F00D0EB7EC01F00A0EB7EC01F050
:10399000170EF76E260EF66EAFEC01F00D0EB7ECBB
:1039A00001F00A0EB7EC01F0170EF76E5A0EF66E24
:1039B000AFEC01F00D0EB7EC01F00A0EB7EC01F020
:1039C000170EF76E740EF66EAFEC01F00D0EB7EC3D
:1039D00001F00A0EB7EC01F0170EF76E880EF66EC6
:1039E000AFEC01F00D0EB7EC01F00A0EB7EC01F0F0
:1039F000170EF76EB00EF66EAFEC01F00D0EB7ECD1
:103A000001F00A0EB7EC01F0170EF76EC20EF66E5B
:103A1000AFEC01F00D0EB7EC01F00A0EB7EC01F0BF
:103A2000170EF76EEA0EF66EAFEC01F00D0EB7EC66
:103A300001F00A0EB7EC01F0180EF76E220EF66ECA
:103A4000AFEC01F00D0EB7EC01F00A0EB7EC01F08F
:103A5000180EF76E400EF66EAFEC01F00D0EB7ECDF
:103A600001F00A0EB7EC01F0180EF76E620EF66E5A
:103A7000AFEC01F00D0EB7EC01F00A0EB7EC01F05F
:103A8000180EF76E820EF66EAFEC01F00D0EB7EC6D
:103A900001F00A0EB7EC01F0180EF76E9A0EF66EF2
:103AA000AFEC01F00D0EB7EC01F00A0EB7EC01F02F
:103AB000180EF76EB40EF66EAFEC01F00D0EB7EC0B
:103AC00001F00A0EB7EC01F0180EF76ED20EF66E8A
:103AD000AFEC01F00D0EB7EC01F00A0EB7EC01F0FF
:103AE000180EF76EF00EF66EAFEC01F00D0EB7EC9F
:103AF00001F00A0EB7EC01F0190EF76E180EF66E13
:103B0000AFEC01F00D0EB7EC01F00A0EB7EC01F0CE
:103B100063EF25F04E0EB15D37E1000E9BB1010E53
:103B2000010AD8B49B91D8A49B81190EF76E420E5E
:103B3000F66EAFEC01F09B3110E34C0EB7EC01F0E8
:103B4000430EB7EC01F0440EB7EC01F00D0EB7ECEC
:103B500001F00A0EB7EC01F00FD04C0EB7EC01F0FB
:103B6000450EB7EC01F0440EB7EC01F00D0EB7ECCA
:103B700001F00A0EB7EC01F0AA6A1E0EA96E9B5165
:103B8000CFEC01F063EF25F0590EB15D3CE1000E82
:103B90009AB1010E010AD8B49A91D8A49A81450E1F
:103BA000B7EC01F0630EB7EC01F0680EB7EC01F072
:103BB0006F0EB7EC01F0200EB7EC01F09A310DE377
:103BC0004F0EB7EC01F04E0EB7EC01F00D0EB7EC56
:103BD00001F00A0EB7EC01F00ED04F0EB7EC01F079
:103BE000460EB7EC01F0B7EC01F00D0EB7EC01F0AA
:103BF0000A0EB7EC01F0AA6A0F0EA96E9A51CFEC2B
:103C000001F063EF25F0510EB15DD8A4AAD001EE0A
:103C100098F010EEF6F0020EF36E030E2EEC03F0A9
:103C2000EF6A190EF76E500EF66E01EE98F042EC48
:103C300003F00BE10301040E556FAA6A110EA96E81
:103C40005551CFEC01F0000149D0190EF76E540E1A
:103C5000F66E01EE98F042EC03F00BE10301140E56
:103C6000556FAA6A110EA96E5551CFEC01F00001F3
:103C700035D001EE98F0EECFF3FFEFCFF4FFF35025
:103C8000310AF41002E0000E01D0010E3B6E190E55
:103C9000F76E580EF66E01EE98F04BEC03F03B1207
:103CA0000BE00301020E556FAA6A110EA96E555161
:103CB000CFEC01F0000112D0190EF76E5C0EF66E1B
:103CC00001EE98F042EC03F009E103010A0E556F92
:103CD000AA6A110EA96E5551CFEC01F0030155519E
:103CE0000FEC09F035C039F034C038F033C037F08C
:103CF00032C036F0356A346A336A800E326E02ECB6
:103D000008F035C0AFF034C0AEF033C0ADF032C013
:103D1000ACF0190EF76E600EF66EAFEC01F0040E0B
:103D2000016EAFC029F0AEC028F0ADC027F0ACC026
:103D300026F0010EA7EC00F0200EB7EC01F0640EA7
:103D4000B7EC01F0650EB7EC01F0670EB7EC01F0CF
:103D50000D0EB7EC01F00A0EB7EC01F0000163EFB5
:103D600025F05A0EB15D41E1000E9AB7010E010A2D
:103D7000D8B49A97D8A49A87190EF76E720EF66E79
:103D8000AFEC01F09A51E8A616D0730EB7EC01F033
:103D90006F0EB7EC01F0750EB7EC01F0740EB7ECD6
:103DA00001F0680EB7EC01F00D0EB7EC01F00A0E51
:103DB000B7EC01F012D06E0EB7EC01F06F0EB7EC5D
:103DC00001F0720EB7EC01F0640EB7EC01F00D0ECD
:103DD000B7EC01F00A0EB7EC01F0AA6A0F0EA96E5B
:103DE0009A51CFEC01F063EF25F0260EB15D23E18F
:103DF0005A0E665C03E1B40E666E02D05A0E666E11
:103E0000190EF76E840EF66EAFEC01F0040E016E23
:103E1000030E076E66506DEC00F00D0EB7EC01F06E
:103E20000A0EB7EC01F0AA6A0E0EA96E6650CFEC2E
:103E300001F063EF25F04A0EB15DD8A494D0190EBD
:103E4000F76E9A0EF66EAFEC01F0F7510B6E4E0E58
:103E50000B5C0FE13A0EB7EC01F0200EB7EC01F06D
:103E60006F0EB7EC01F0660EB7EC01F0B7EC01F0A5
:103E70009A9BF7510B6E460E0B5C08E1190EF76E1C
:103E8000A20EF66EAFEC01F09A899A8BF7510B6E89
:103E9000440E0B5C08E1190EF76EAE0EF66EAFEC39
:103EA00001F09A999A8BF7510301BD6F000171ECF3
:103EB0004BF045AE49D001EE98F010EEF6F0020E50
:103EC000F36E050E2EEC03F0EF6A01EE98F020EC95
:103ED00000F00301856F1CC086F3190EF76EC00E4B
:103EE000F66EAFEC01F0040E016E076A86C31CF09B
:103EF00085C31BF06FEC00F0AA6A1C0EA96E86C386
:103F000014F085C313F0186A0A0E176E61EC02F004
:103F1000266E14C027F02650CFEC01F02750CFECCE
:103F200001F0166A070E156EA10E146E200E136EA8
:103F300085C31BF086C31CF01D6A1E6A36EC02F0B6
:103F400014C084F313C083F300010D0EB7EC01F02D
:103F50000A0EB7EC01F0AA6A0F0EA96E9A51CFECC7
:103F600001F063EF25F0540EB15DD8A4AED0F75147
:103F70000301BD6F000171EC4BF045AEA3D001EE23
:103F800098F010EEF6F0020EF36E050E2EEC03F034
:103F9000EF6A01EE98F020EC00F08A6F1CC08BF005
:103FA000190EF76ECE0EF66EAFEC01F0040E016E38
:103FB000076A8BC01CF08AC01BF06FEC00F00D0E7E
:103FC000B7EC01F00A0EB7EC01F0190EF76EE00E37
:103FD000F66EAFEC01F00D0EB7EC01F00A0EB7EC87
:103FE00001F0B951120AC00ED8B4B81902E1000E9E
:103FF00001D0010E3B6EB951250A800ED8B4B81914
:1040000002E1000E01D0010E3B16B9514B0AB81166
:1040100002E1000E01D0010E3B16B951960AB8110B
:1040200002E1000E01D0010E3B16B951E10AB811B0
:1040300002E1000E01D0010E3B160CE01A0EF76EE5
:104040000A0EF66EAFEC01F00D0EB7EC01F00A0EA1
:10405000B7EC01F0AA6A1F0EA96E8A51CFEC01F0ED
:104060008B51CFEC01F01A0EF76E540EF66EAFECDA
:1040700001F00D0EB7EC01F00A0EB7EC01F00B0EDB
:10408000086EB80E026E90EC01F01CE3A96FA99BBC
:104090009A3103E3A951B7EC01F0590EA95D12E181
:1040A0001A0EF76E760EF66EAFEC01F00D0EB7EC51
:1040B00001F00A0EB7EC01F08BC0B9F08AC0B8F07D
:1040C00094EC43F0B16B63EF25F0250EB15D38E160
:1040D000000E9AB3010E010AD8B49A93D8A49A8319
:1040E0001A0EF76E8E0EF66EAFEC01F09A51E8B232
:1040F0000DD04F0EB7EC01F04E0EB7EC01F00D0EE7
:10410000B7EC01F00A0EB7EC01F00ED04F0EB7EC91
:1041100001F0460EB7EC01F0B7EC01F00D0EB7EC74
:1041200001F00A0EB7EC01F0800E016E10EC00F009
:10413000AA6A0F0EA96E9A51CFEC01F063EF25F039
:104140002A0EB15D38E101EE98F010EEF6F0020EA5
:10415000F36E030E2EEC03F0EF6A04EE15F011EE91
:1041600098F0060E27EC03F0A2EC4AF0AEC3B3F0D1
:10417000ADC3B2F0B351E8AE02D0000E01D0010ED3
:104180003B6EB351E8BE07D0B35303E1B2515A08B6
:1041900002E2000E01D0010E3B16000109E0B2C0A0
:1041A00059F3AA6A100EA96E03015951CFEC01F020
:1041B000000163EF25F0460EB15DD8A49CD0F75105
:1041C0000B6E3F0E0B5C30E16F50735C266E7050CF
:1041D0007458276E27C022F026C021F055C31BF06B
:1041E0001C6A78EC02F0906F14C091F09A51E8A626
:1041F00004D0B40E905F000E915B1A0EF76E9C0E09
:10420000F66EAFEC01F0040E016E030E076E91C066
:104210001CF090C01BF06FEC00F00D0EB7EC01F03D
:104220000A0EB7EC01F065D0F7510301BD6F000134
:1042300071EC4BF045AE3FD001EE98F010EEF6F089
:10424000020EF36E030E2EEC03F0EF6A04EE15F08F
:1042500011EE98F0060E27EC03F0A2EC4AF0AEC384
:10426000B3F0ADC3B2F0B351E8BE23D0B251B31135
:1042700020E0B3C074F0B2C073F09A51E8A604D045
:10428000B40E7326000E7422735003015503F3CF4E
:1042900026F0F4CF27F074505503F350272655AF7E
:1042A00002D07350275E6F502624736E7050272003
:1042B000746E000109D0F7510B6E210E0B5C04E106
:1042C0004BC074F04AC073F0AA6A0C0EA96E73500A
:1042D000CFEC01F07450CFEC01F01A0EF76EB20E75
:1042E000F66EAFEC01F00D0EB7EC01F00A0EB7EC74
:1042F00001F063EF25F0230EB15D2CE1000E9AB5BD
:10430000010E010AD8B49A95D8A49A851A0EF76EB0
:10431000BE0EF66EAFEC01F09A51E8B40AD0410E31
:10432000B7EC01F00D0EB7EC01F00A0EB7EC01F09E
:1043300009D0420EB7EC01F00D0EB7EC01F00A0EF9
:10434000B7EC01F0AA6A0F0EA96E9A51CFEC01F0FA
:1043500063EF25F0490EB15DD8A46CEF24F00D0E8B
:10436000B7EC01F00A0EB7EC01F01A0EF76ECA0EA8
:10437000F66EAFEC01F00D0EB7EC01F00A0EB7ECE3
:1043800001F01A0EF76EEC0EF66EAFEC01F0040EB3
:10439000016E076A70C022F06FC021F055C31BF098
:1043A0001C6A78EC02F01B6E14C01CF06FEC00F07D
:1043B000200EB7EC01F0640EB7EC01F0650EB7EC1F
:1043C00001F0670EB7EC01F00D0EB7EC01F00A0E2C
:1043D000B7EC01F01B0EF76E000EF66EAFEC01F0BD
:1043E000040E016E076A72C022F071C021F055C33D
:1043F0001BF01C6A78EC02F01B6E14C01CF06FEC12
:1044000000F0200EB7EC01F0640EB7EC01F0650E81
:10441000B7EC01F0670EB7EC01F00D0EB7EC01F050
:104420000A0EB7EC01F06F50735C266E7050745832
:10443000276E27C022F026C021F055C31BF01C6A4E
:1044400078EC02F0906F14C091F09A51E8A604D075
:10445000B40E905F000E915B1B0EF76E160EF66E9B
:10446000AFEC01F0040E016E076A91C01CF090C021
:104470001BF06FEC00F0200EB7EC01F0640EB7EC0F
:1044800001F0650EB7EC01F0670EB7EC01F00D0E10
:10449000B7EC01F00A0EB7EC01F01B0EF76E340E0C
:1044A000F66EAFEC01F0040E016E66506CEC00F09D
:1044B000200EB7EC01F0640EB7EC01F0650EB7EC1E
:1044C00001F0670EB7EC01F00D0EB7EC01F00A0E2B
:1044D000B7EC01F01B0EF76E540EF66EAFEC01F068
:1044E000040E016E030159516CEC00F0200EB7EC84
:1044F00001F0640EB7EC01F0650EB7EC01F0670E49
:10450000B7EC01F00D0EB7EC01F00A0EB7EC01F0BC
:104510001B0EF76E760EF66EAFEC01F000019A51AD
:10452000E8A209D04F0EB7EC01F0460EB7EC01F04F
:10453000B7EC01F006D04F0EB7EC01F04E0EB7EC21
:1045400001F00D0EB7EC01F00A0EB7EC01F01B0EF6
:10455000F76E8A0EF66EAFEC01F0040E016E030EDC
:10456000076E68C022F067C021F055C31BF01C6ABB
:1045700078EC02F01B6E14C01CF06FEC00F0200E03
:10458000B7EC01F0450EB7EC01F04C0EB7EC01F0C2
:104590003A0EB7EC01F0200EB7EC01F0030E076EF7
:1045A0006AC022F069C021F055C31BF01C6A78EC88
:1045B00002F01B6E14C01CF06FEC00F00D0EB7EC97
:1045C00001F00A0EB7EC01F01A0EF76EBE0EF66E91
:1045D000AFEC01F09A51E8B404D0410EB7EC01F011
:1045E00003D0420EB7EC01F00D0EB7EC01F00A0E4D
:1045F000B7EC01F01B0EF76E9A0EF66EAFEC01F001
:104600009A51E8B60DD04E0EB7EC01F06F0EB7EC34
:1046100001F0720EB7EC01F0640EB7EC01F00FD0B0
:10462000530EB7EC01F06F0EB7EC01F0750EB7EC5E
:1046300001F0740EB7EC01F0680EB7EC01F00D0E4E
:10464000B7EC01F00A0EB7EC01F0190EF76ECE0EC2
:10465000F66EAFEC01F0040E016E076AB9C01CF0F3
:10466000B8C01BF06FEC00F00D0EB7EC01F00A0EB5
:10467000B7EC01F01B0EF76EAA0EF66EAFEC01F070
:104680009A3107E34F0EB7EC01F04E0EB7EC01F094
:1046900008D04F0EB7EC01F0460EB7EC01F0B7ECC6
:1046A00001F00D0EB7EC01F00A0EB7EC01F01B0E95
:1046B000F76EBA0EF66EAFEC01F09A51E8AA11D07F
:1046C0009A51E8A807D01B0EF76EC40EF66EAFEC39
:1046D00001F006D01B0EF76ECE0EF66EAFEC01F0B9
:1046E00008D04F0EB7EC01F0460EB7EC01F0B7EC76
:1046F00001F0000E9ABB010E3B6E000E9AB9010E3E
:104700003B161EE00D0EB7EC01F00A0EB7EC01F0FF
:104710001B0EF76EDE0EF66EAFEC01F0040E016EAE
:10472000076A86C31CF085C31BF06FEC00F0200EF7
:10473000B7EC01F0480EB7EC01F07A0EB7EC01F0DF
:104740000D0EB7EC01F00A0EB7EC01F01B0EF76E80
:10475000F20EF66EAFEC01F0030155510FEC09F0CB
:1047600035C039F034C038F033C037F032C036F0DD
:10477000356A346A336A800E326E02EC08F035C056
:10478000AFF034C0AEF033C0ADF032C0ACF0040EC8
:10479000016EAFC029F0AEC028F0ADC027F0ACC0AC
:1047A00026F0010EA7EC00F0200EB7EC01F0640E2D
:1047B000B7EC01F0650EB7EC01F0670EB7EC01F055
:1047C0000D0EB7EC01F00A0EB7EC01F01B0EF76E00
:1047D000FE0EF66EAFEC01F000019B310AE34C0EC9
:1047E000B7EC01F0430EB7EC01F0440EB7EC01F06A
:1047F00009D04C0EB7EC01F0450EB7EC01F0440EB9
:10480000B7EC01F00D0EB7EC01F00A0EB7EC01F0B9
:104810001C0EF76E0E0EF66EAFEC01F0040E016E7C
:104820003DC329F03CC328F03BC327F03AC326F030
:10483000050EA7EC00F01C0EF76E1A0EF66EAFEC2C
:1048400001F0040E016E41C329F040C328F03FC3BC
:1048500027F03EC326F0050EA7EC00F00D0EB7ECD6
:1048600001F00A0EB7EC01F01C0EF76E280EF66E82
:10487000AFEC01F0040E016E8EC329F08DC328F059
:104880008CC327F08BC326F0010EA7EC00F00D0EB1
:10489000B7EC01F00A0EB7EC01F01C0EF76E3C0EFF
:1048A000F66EAFEC01F0040E016E076A8AC31BF0CE
:1048B0001C6A6FEC00F01C0EF76E440EF66EAFEC47
:1048C00001F0076A89C31BF01C6A6FEC00F0000E50
:1048D000B7EC01F0B16BF7D03C0EB15D36E11C0EC8
:1048E000F76E4C0EF66EAFEC01F00D0EB7EC01F06A
:1048F0000A0EB7EC01F0AAEC01F0A96FA99B9A315E
:1049000003E3A951B7EC01F0590EA95D1DE131ECAB
:1049100037F042BE0DD01C0EF76E5A0EF66EAFEC9D
:1049200001F00D0EB7EC01F00A0EB7EC01F00CD05F
:104930001C0EF76E700EF66EAFEC01F00D0EB7ECBC
:1049400001F00A0EB7EC01F0BED05E0EB15D36E1AB
:104950001C0EF76E4C0EF66EAFEC01F00D0EB7ECC0
:1049600001F00A0EB7EC01F0AAEC01F0A96FA99BC7
:104970009A3103E3A951B7EC01F0590EA95D1DE18D
:10498000D8EC37F043B00DD01C0EF76E8A0EF66EE1
:10499000AFEC01F00D0EB7EC01F00A0EB7EC01F030
:1049A0000CD01C0EF76EA20EF66EAFEC01F00D0EE1
:1049B000B7EC01F00A0EB7EC01F085D05B0EB15DEB
:1049C00035E101EE98F010EEF6F0020EF36E080EEF
:1049D0002EEC03F0EF6A04EE1CF011EE98F0140ECA
:1049E00027EC03F0C6EC4AF0B3C33DF3B2C33CF38B
:1049F000B1C33BF3B0C33AF31C0EF76EBE0EF66EB6
:104A0000AFEC01F0040E016E3DC329F03CC328F069
:104A10003BC327F03AC326F0050EA7EC00F00D0EBD
:104A2000B7EC01F00A0EB7EC01F04DD05D0EB15DB0
:104A300035E101EE98F010EEF6F0020EF36E090E7D
:104A40002EEC03F0EF6A04EE1CF011EE98F0140E59
:104A500027EC03F0C6EC4AF0B3C341F3B2C340F312
:104A6000B1C33FF3B0C33EF31C0EF76ECA0EF66E31
:104A7000AFEC01F0040E016E41C329F040C328F0F1
:104A80003FC327F03EC326F0050EA7EC00F00D0E45
:104A9000B7EC01F00A0EB7EC01F015D09A3113E330
:104AA0003F0EB7EC01F03E0EB7EC01F000EEF6F071
:104AB000EE5003E0B7EC01F0FBD70D0EB7EC01F0C0
:104AC0000A0EB7EC01F000EEF6F0EF6AB16B42BCF3
:104AD0001DD16F504A5C4E6E70504B584F6E7150E6
:104AE0004C5C506E72504D58516E000E45B0010E28
:104AF0003B6EC6514E5CC7514F584F50C719D8B086
:104B0000800A02E6000E01D0010E3B1603E09396E8
:104B10008A96449C000E45B2010E3B6E4FBE05D0F6
:104B20004E504F1002E0000E01D0010E3B1603E084
:104B300093988A98449C000E42B0010E3B6E010E81
:104B400042BE000E3B16D8B440D04A505E5C4B507B
:104B50005F584B505F18D8B0800A0CE681A604D08D
:104B600093968A96E7EC43F04590458293988A881D
:104B700095968C865E504A5C5F504B584B505F1840
:104B8000D8B0800A0CE681A804D093988A98E7EC04
:104B900043F04592458093968A8695968C865F5021
:104BA0004B5C03E15E504A5C02E0000E01D0010E56
:104BB0003B6E000E42BC010E3B12000106E09396D4
:104BC0008A9693988A984290449C010E9AB3000E5C
:104BD0003B6E49AE02D0000E01D0010E3B1648508C
:104BE000C85D4950C9594950C919D8B0800A02E670
:104BF000000E01D0010E3B16D8B475D0000E45B49E
:104C0000010E3B6EC851505CC95151585150C919E1
:104C1000D8B0800A02E6000E01D0010E3B1603E078
:104C2000939A8A9A449C000E45B6010E3B6E51BE83
:104C300005D05050511002E0000E01D0010E3B167D
:104C400003E0939C8A9C449C010E43B0000E3B6E93
:104C5000000E42B2010E3B16D8B445D071504C5CE8
:104C6000506E72504D58516E5050485C51504958DA
:104C700051504918D8B0800A0CE681AA04D0939A02
:104C80008A9AE7EC43F045944586939C8A8C9596E6
:104C90008C864850505C4950515851504918D8B0F2
:104CA000800A0CE681AC04D0939C8A9CE7EC43F02C
:104CB00045964584939A8A8A95968C864950515C8C
:104CC00003E14850505C02E0000E01D0010E3B6E43
:104CD000000E42BC010E3B12000105E0939C8A9C31
:104CE000939A8A9A4292010E42B4000E3B6E010ED4
:104CF00042B6000E3B16010E42B0000E3B16010EEE
:104D000042B2000E3B1602E095968C9645EF13F0EA
:104D10006F504A5C4E6E70504B584F6E71504C5CE9
:104D2000506E72504D58516E4FBE02D0000E01D0E1
:104D3000010E3B6E4E50C65D4F50C7594F50C719BC
:104D4000D8B0800A02E7000E01D0010E3B1202E04B
:104D5000838201D0839251BE02D0000E01D0010E99
:104D60003B6E5050C85D5150C9595150C919D8B007
:104D7000800A02E7000E01D0010E3B1202E08380A0
:104D800001D083909A51E8A614D0C4514E26C55143
:104D90004F22C6514E5CC7514F584F50C719D8B01B
:104DA000800A06E7C6514E5C4E6EC7514F584F6E93
:104DB00015D04FAE04D0C6514E26C7514F22C65112
:104DC0004E5CC7514F584F50C719D8B0800A06E7FC
:104DD000C6514E5C4E6EC7514F584F6E9B3102E329
:104DE00004D802D075EC2AF012009A51E8B2B0EF64
:104DF00029F043B077D143BE1CD1FE0E5014526E41
:104E0000FF0E5114536E53AE8ED0800E016E19EC0E
:104E100000F0450E43EC01F04C0E43EC01F03A0E6D
:104E200043EC01F0200E43EC01F02D0E43EC01F0B9
:104E300053C00CF052C00BF00CAE03D00B6CE86A00
:104E40000C56CA510B5CCB510C580C50CB19D8B036
:104E5000800A04E6200E43EC01F01BD053C00CF096
:104E600052C00BF00CAE03D00B6CE86A0C560CC0B1
:104E700022F00BC021F0CBC01CF0CAC01BF078ECB4
:104E800002F09D6F800E016E010E076E9D516DEC5C
:104E900000F0800E016E010E076E53C00CF052C080
:104EA0000BF00CAE03D00B6CE86A0C560CC022F071
:104EB0000BC021F055C31BF01C6A78EC02F01B6E8E
:104EC00014C01CF06FEC00F02E0E43EC01F053C048
:104ED0000CF052C00BF00CAE03D00B6CE86A0C5611
:104EE0000CC022F00BC021F055C31BF01C6A78ECFB
:104EF00002F017C09DF09D510A0DF3CF26F0F4CFBC
:104F000027F027C014F026C013F0186A55C317F015
:104F100061EC02F09D6F800E016E010E076E9D51D7
:104F20006DEC00F085D0800E016E19EC00F0450E9E
:104F300043EC01F04C0E43EC01F03A0E43EC01F06F
:104F4000200E43EC01F0CC51525CCD5153585350DC
:104F5000CD19D8B0800A04E6200E43EC01F012D03F
:104F600053C022F052C021F0CDC01CF0CCC01BF0C9
:104F700078EC02F09D6F800E016E010E076E9D5160
:104F80006DEC00F0CA51525CCB5153585350CB19C1
:104F9000D8B0800A04E6200E43EC01F012D053C0D2
:104FA00022F052C021F0CBC01CF0CAC01BF078EC3C
:104FB00002F09D6F800E016E010E076E9D516DEC2B
:104FC00000F0800E016E010E076E53C022F052C039
:104FD00021F055C31BF01C6A78EC02F01B6E14C064
:104FE0001CF06FEC00F02E0E43EC01F053C022F0E9
:104FF00052C021F055C31BF01C6A78EC02F017C0B8
:105000009DF09D510A0DF3CF26F0F4CF27F027C075
:1050100014F026C013F0186A55C317F061EC02F0C3
:105020009D6F800E016E010E076E9D516DEC00F0BC
:1050300058D0356A346A200E336E820E326E37C312
:1050400039F036C338F035C337F034C336F068EC86
:1050500008F0B6EC08F0526E33C053F0800E016ECB
:1050600019EC00F0450E43EC01F04C0E43EC01F05E
:105070003A0E43EC01F0200E43EC01F043EC01F05A
:1050800037C335F036C334F035C333F034C332F0B0
:10509000396A386A200E376E820E366EB8EC06F02A
:1050A000010803E0200E43EC01F0800E016E076A58
:1050B00053C022F052C021F01C6A0A0E1B6E78EC1D
:1050C00002F01B6E14C01CF06FEC00F02E0E43ECCF
:1050D00001F0010E076E53C01CF052C01BF06FECC4
:1050E00000F00AD0800E016E19EC00F01C0EF76E75
:1050F000D60EF66E3BEC01F08AAC03D0000E43EC0A
:1051000001F08AAA03D0010E43EC01F0010E8ABA25
:10511000000E3B6E010E8ABC000E3B1603E0200E13
:1051200043EC01F08AA803D0030E43EC01F08AA6F9
:1051300003D0020E43EC01F0010E8AB6000E3B6E66
:10514000010E8AB8000E3B1603E0200E43EC01F07E
:1051500043BE98D042BE8FD043BE07D0FE0E4E1441
:10516000546EFF0E4F14556E04D047C055F046C024
:1051700054F0410E43EC01F05A0E43EC01F03A0EAC
:1051800043EC01F0200E43EC01F0CC51545CCD51C6
:1051900055585550CD19D8B0800A04E6200E43EC7E
:1051A00001F012D055C022F054C021F0CDC01CF047
:1051B000CCC01BF078EC02F09D6F800E016E010EEA
:1051C000076E9D516DEC00F0CA51545CCB5155589F
:1051D0005550CB19D8B0800A04E6200E43EC01F0FC
:1051E00012D055C022F054C021F0CBC01CF0CAC070
:1051F0001BF078EC02F09D6F800E016E010E076EC1
:105200009D516DEC00F0800E016E010E076E55C0D1
:1052100022F054C021F055C31BF01C6A78EC02F058
:105220001B6E14C01CF06FEC00F02E0E43EC01F06E
:1052300055C022F054C021F055C31BF01C6A78EC15
:1052400002F017C09DF09D510A0DF3CF26F0F4CF68
:1052500027F027C014F026C013F0186A55C317F0C2
:1052600061EC02F09D6F800E016E010E076E9D5184
:105270006DEC00F006D01C0EF76EE00EF66E3BEC07
:1052800001F067D0356A346A200E336E820E326EBA
:1052900033C339F032C338F031C337F030C336F09E
:1052A00068EC08F0B6EC08F0546E33C055F0410ECF
:1052B00043EC01F05A0E43EC01F03A0E43EC01F0DE
:1052C000200E43EC01F033C335F032C334F031C368
:1052D00033F030C332F0396A386A480E376E850EC3
:1052E000366EB8EC06F0010803E0200E43EC01F046
:1052F00033C335F032C334F031C333F030C332F04E
:10530000396A386A200E376E820E366EB8EC06F0B7
:10531000010803E0200E43EC01F0800E016E076AE5
:1053200055C022F054C021F01C6A0A0E1B6E78ECA6
:1053300002F01B6E14C01CF06FEC00F02E0E43EC5C
:1053400001F0010E076E55C01CF054C01BF06FEC4D
:1053500000F01C0EF76EEA0EF66E3BEC01F0C4D0C6
:1053600042BEB2D043BE07D0FE0E4E14546EFF0EA6
:105370004F14556E04D047C055F046C054F0800E0F
:10538000016E19EC00F01D0EF76E000EF66E3BEC90
:1053900001F0CC51545CCD5155585550CD19D8B071
:1053A000800A04E6200E43EC01F012D055C022F032
:1053B00054C021F0CDC01CF0CCC01BF078EC02F042
:1053C0009D6F800E016E010E076E9D516DEC00F019
:1053D000CA51545CCB5155585550CB19D8B0800A9E
:1053E00004E6200E43EC01F012D055C022F054C068
:1053F00021F0CBC01CF0CAC01BF078EC02F09D6F0E
:10540000800E016E010E076E9D516DEC00F0800E56
:10541000016E010E076E55C022F054C021F055C335
:105420001BF01C6A78EC02F01B6E14C01CF06FECD1
:1054300000F02E0E43EC01F055C022F054C021F0D4
:1054400055C31BF01C6A78EC02F017C09DF09D510B
:105450000A0DF3CF26F0F4CF27F027C014F026C0B2
:1054600013F0186A55C317F061EC02F09D6F800EBF
:10547000016E010E076E9D516DEC00F0200E43ECA5
:1054800001F0640E43EC01F0650E43EC01F0670E91
:1054900043EC01F0200E43EC01F08AA803D0030E88
:1054A00043EC01F08AA603D0020E43EC01F0010E9A
:1054B0008AB6000E3B6E010E8AB8000E3B1603E062
:1054C000200E43EC01F00AD0800E016E19EC00F0C2
:1054D0001D0EF76E0A0EF66E3BEC01F01D0EF76E18
:1054E000200EF66E3BEC01F012000EEC00F06F5057
:1054F0004A5C4E6E70504B584F6E71504C5C506E03
:1055000072504D58516E9A51E8A614D0C4514E268F
:10551000C5514F22C6514E5CC7514F584F50C71905
:10552000D8B0800A06E7C6514E5C4E6EC7514F5840
:105530004F6E15D04FAE04D0C6514E26C7514F22E4
:10554000C6514E5CC7514F584F50C719D8B0800A4A
:1055500006E7C6514E5C4E6EC7514F584F6E449A87
:1055600051BE448A51C00CF050C00BF00CAE03D0B9
:105570000B6CE86A0C560CC022F00BC021F055C32E
:105580001BF01C6A78EC02F0626E14C063F063C01A
:1055900014F062C013F0020E2CEC02F09C6F00EECF
:1055A000DAF09C51EBCF0BF00BC0D4F063C014F0D9
:1055B00062C013F0010E2CEC02F09C6F00EEDAF0EA
:1055C0009C51EBCF0BF00BC0D5F063C014F062C060
:1055D00013F0000E2CEC02F09C6F00EEDAF09C5100
:1055E000EBCF0BF00BC0D6F04FC00CF04EC00BF061
:1055F0000CAE03D00B6CE86A0C560CC022F00BC04A
:1056000021F055C31BF01C6A78EC02F0606E14C0E8
:1056100061F061C014F060C013F0020E2CEC02F0D7
:105620009C6F00EEDAF09C51EBCF0BF00BC0D7F083
:1056300061C014F060C013F0010E2CEC02F09C6FFE
:1056400000EEDAF09C51EBCF0BF00BC0D8F061C04C
:1056500014F060C013F0000E2CEC02F09C6F00EE12
:10566000DAF09C51EBCF0BF00BC0D9F063BE05D044
:10567000635207E1640E625C04E2E4C00BF00BC00D
:10568000D4F0000163BE05D0635207E10A0E625CEC
:1056900004E2E4C00BF00BC0D5F0000161BE05D000
:1056A000615207E1640E605C04E2E4C00BF00BC0E1
:1056B000D7F0000161BE05D0615207E10A0E605CBF
:1056C00004E2E4C00BF00BC0D8F0000144AA04D0FF
:1056D000F4C00BF00BC0D4F081AC07D0D4510F6EE6
:1056E000FE0E0F140B6E0BC0D4F081AA07D0D6515A
:1056F0000F6EFE0E0F140B6E0BC0D6F081A807D0F4
:10570000D7510F6EFE0E0F140B6E0BC0D7F081A693
:1057100007D0D9510F6EFE0E0F140B6E0BC0D9F0CF
:1057200083A007D0D5510F6EFE0E0F140B6E0BC069
:10573000D5F083A207D0D8510F6EFE0E0F140B6E5A
:105740000BC0D8F09A51E8A20DD0E4C00BF00BC00A
:10575000D4F0E4C00BF00BC0D5F0E4C00BF00BC0EC
:10576000D6F00ED043A00CD0EAC00BF00BC0D4F0A2
:10577000F1C00BF00BC0D5F0F1C00BF00BC0D6F0B0
:1057800042AE0CD0EAC00BF00BC0D7F0F1C00BF06A
:105790000BC0D8F0F1C00BF00BC0D9F0840E026E34
:1057A000020E086E840E036E010E046E050E096E65
:1057B000D451136EEBEC01F0840E026E020E086EF3
:1057C000840E036E010E046E050E096ED551136E24
:1057D000EBEC01F0840E026E020E086E840E036E76
:1057E000010E046E050E096ED651136EEBEC01F03E
:1057F000840E026E020E086E840E036E010E046E9D
:10580000050E096ED751136EEBEC01F0840E026E9B
:10581000020E086E840E036E010E046E050E096EF4
:10582000D851136EEBEC01F0840E026E020E086E7E
:10583000840E036E010E046E050E096ED951136EAF
:10584000EBEC01F096948D8496948D941200449A1A
:105850009551E8AE01D0448A95C00CF094C00BF08D
:105860000CAE03D00B6CE86A0C560CC022F00BC0D7
:1058700021F055C31BF01C6A78EC02F0946F14C041
:1058800095F095C014F094C013F0020E2CEC02F0C9
:105890009C6F00EEDAF09C51EBCF0BF00BC0D7F011
:1058A00095C014F094C013F0010E2CEC02F09C6F24
:1058B00000EEDAF09C51EBCF0BF00BC0D8F095C0A6
:1058C00014F094C013F0000E2CEC02F09C6F00EE6C
:1058D000DAF09C51EBCF0BF00BC0D9F044AA04D006
:1058E000F4C00BF00BC0D7F0D5EF40F093968A963A
:1058F00093988A98939C8A9C939A8A9A95968C9668
:1059000049C0BFF048C0BEF047C0BDF046C0BCF0C3
:10591000B76B010EB66FB7530CE1330EB65D09E2FB
:10592000010E14EC02F06AEC40F0B62B000EB72327
:10593000F2E382B23AD0010E42B4000E3B6E010E89
:1059400042B6000E3B1608E0000E42BC010E010AF2
:10595000D8B4429CD8A4428C42904292429442963F
:10596000429E43900301516B526B00EEF6F0EF6ADA
:10597000449C42BC828042AC82900001BB6BBA6BFB
:1059800082B213D0BA4BBB2B030E146E200E22EC46
:1059900002F0050EBB5D06E303E1DD0EBA5D02E336
:1059A000000104D06AEC40F0EBD712008290429CD8
:1059B000976B839283900EEC00F0800E016E19ECD1
:1059C00000F01D0EF76E360EF66E3BEC01F01D0E6C
:1059D000F76E4C0EF66E3BEC01F0F4C00BF00BC012
:1059E000D4F0F4C00BF00BC0D5F0F4C00BF00BC03A
:1059F000D6F0F4C00BF00BC0D7F0F4C00BF00BC026
:105A0000D8F0F4C00BF00BC0D9F0D5EC40F082A276
:105A1000FED70301140E546F4FC022F04EC021F088
:105A200055C31BF01C6A78EC02F05A6E14C05BF090
:105A30005B5003015503F3CF5BF05A505503F3CF8E
:105A40005AF0F4505B2655AF02D05A505B5E51C0FD
:105A50005DF050C05CF068C06CF067C06BF06AC06D
:105A60006EF069C06DF070C076F06FC075F072C0F6
:105A700078F071C077F06F50735C796E7050745825
:105A80007A6E00019A51E8A606D0C451795C796E0D
:105A9000C5517A587A6E43829AA1439243849AA35D
:105AA0004394438A9AA5439A66C0B0F043869AA766
:105AB000439643889AA94398438C9AAB439C44806D
:105AC00043AE449055C37DF059C37BF07C6A428855
:105AD0009AAD4298428A9AAF429AB9C08BF0B8C048
:105AE0008AF03DC381F03CC380F03BC37FF03AC3F2
:105AF0007EF041C385F040C384F03FC383F03EC3D2
:105B000082F043C387F042C386F0458A9BA1459A41
:105B1000B05103015503F4CFC9F0F3CFC8F086C3E9
:105B200089F085C388F0000180BC1CD0140E14ECF1
:105B300002F080BC16D09607010E965D02E21A0EA6
:105B4000966F0F0E965D0AE1010E43BC000E3B6E90
:105B5000010E43B8000E3B1201E096070301140E3C
:105B6000546F000180BE1CD0140E14EC02F080BEF5
:105B700016D0962B1B0E965D02E3010E966F0F0E4C
:105B8000965D0AE1010E43BC000E3B6E010E43B868
:105B9000000E3B1201E0962B0301140E546F00011E
:105BA00082B40AD0140E14EC02F082B402D0FF0EBC
:105BB000976F0301140E546F000182B60AD0140EC1
:105BC00014EC02F082B602D0010E976F0301140E9E
:105BD000546F0001010E82B2000E3B6E010E0301F4
:105BE0005453D8A4000E3B120001D8B4B8D10E0E05
:105BF000965D010ED8A4000E3B6E010E82B2000E1F
:105C00003B1606E0439C0301140E546F0001A7D11C
:105C10005BC047F05AC046F05DC049F05CC048F038
:105C2000000E66BEFF0E495C07E049506618D8B00A
:105C3000800A800B1EE003D04850665C1AE2485090
:105C40000001C45D486E4950C559496EC45146268D
:105C5000C5514722C651465CC75147584750C719DE
:105C6000D8B0800A06E7C651465C466EC751475811
:105C7000476E6CC068F06BC067F06EC06AF06DC0B4
:105C800069F076C070F075C06FF078C072F077C0C0
:105C900071F075507924736E76507A20746E9A5133
:105CA000E8A604D0C4517326C55174229A8143A238
:105CB0009A919A8343A49A939A8543AA9A95B0C0DD
:105CC00066F09A8743A69A979A8943A89A999A8BDD
:105CD00043AC9A9B438E44A0439E81C03DF380C059
:105CE0003CF37FC03BF37EC03AF385C041F384C0F0
:105CF00040F383C03FF382C03EF387C043F386C0C6
:105D000042F38BC0B9F08AC0B8F09B8145AA9B9141
:105D10007DC055F303015551B40DF3CFC4F0F4CF5A
:105D2000C5F05551680DF3CFC6F0F4CFC7F00001B0
:105D3000C727665003015503F4CFC9F0F3CFC8F06D
:105D400055510A0DF3CFCAF0F4CFCBF05551640D85
:105D5000F3CFCCF0F4CFCDF07BC059F300019A8D96
:105D600042A89A9D9A8F42AA9A9F89C086F388C0BA
:105D700085F3665003015503F4CFC9F0F3CFC8F0A3
:105D8000AA6A040EA96E6750CFEC01F06850CFEC00
:105D900001F0AA6A060EA96E6950CFEC01F06A50B4
:105DA000CFEC01F0AA6A080EA96E6F50CFEC01F09B
:105DB0007050CFEC01F0AA6A0A0EA96E7150CFECB8
:105DC00001F07250CFEC01F0AA6A0C0EA96E73506C
:105DD000CFEC01F07450CFEC01F0AA6A0E0EA96E60
:105DE0006650CFEC01F0AA6A0F0EA96E00019A511D
:105DF000CFEC01F0AA6A1E0EA96E9B51CFEC01F008
:105E0000AA6A100EA96E03015951CFEC01F0AA6ADB
:105E1000110EA96E03015551CFEC01F0AA6A120EC2
:105E2000A96E03013A51CFEC01F003013B51CFECD5
:105E300001F003013C51CFEC01F003013D51CFECE7
:105E400001F0AA6A160EA96E03013E51CFEC01F0D3
:105E500003013F51CFEC01F003014051CFEC01F0C1
:105E600003014151CFEC01F0AA6A1A0EA96E030199
:105E70004251CFEC01F003014351CFEC01F0AA6A8B
:105E80001F0EA96E0001B851CFEC01F0B951CFEC53
:105E900001F0AA6A1C0EA96E86C314F085C313F024
:105EA000186A0A0E176E61EC02F0266E14C027F015
:105EB0002650CFEC01F02750CFEC01F0166A070E08
:105EC000156EA10E146E200E136E85C31BF086C3D3
:105ED0001CF01D6A1E6A36EC02F014C084F313C075
:105EE00083F394EC43F0800E016E10EC00F0F5ECBF
:105EF00026F082A2FED7000E42B0010E3B6E000ECD
:105F000042B2010E3B1202E095968C869A51E8A6A9
:105F100016D0C45146245E6EC55147205F6E5E5058
:105F2000C65D5F50C7595F50C719D8B0800A06E6F2
:105F3000C6515E5C5E6EC7515F585F6E04D047C04D
:105F40005FF046C05EF047C09AF346C099F35EEC3E
:105F500044F09CC35FF09BC35EF0429C1200010EB4
:105F6000965DD8A450D0975103015503F3CF26F086
:105F7000F4CF27F055AF01D0275E000197AF03D0D3
:105F800003015551275E26505A2627505B220001F7
:105F9000975301E042805A50C65D5B50C7595B5031
:105FA000C719D8B0800A06E6C6515A5C5A6EC75166
:105FB0005B585B6E5BAE04D0C6515A26C7515B225C
:105FC000800E016E19EC00F01D0EF76E620EF66E7B
:105FD0003BEC01F0800E016E030E076E5BC022F0F9
:105FE0005AC021F055C31BF01C6A78EC02F01B6EFE
:105FF00014C01CF06FEC00F0050E43EC01F03BEC1C
:1060000043F0DAEF36F0020E965DD8A450D09751E7
:1060100003015503F3CF26F0F4CF27F055AF01D09D
:10602000275E000197AF03D003015551275E26502C
:106030005C2627505D220001975301E042825C50AC
:10604000C85D5D50C9595D50C919D8B0800A07E6CE
:10605000B05103015503F4CF5DF0F3CF5CF00001C4
:106060005DAE02D05D6A5C6A800E016E19EC00F0D4
:106070001D0EF76E740EF66E3BEC01F0800E016E95
:10608000030E076E5DC022F05CC021F055C31BF00B
:106090001C6A78EC02F01B6E14C01CF06FEC00F070
:1060A000050E43EC01F03BEC43F0DAEF36F0030E63
:1060B000965DD8A449D0975103015503F3CF26F03C
:1060C000F4CF27F055AF01D0275E000197AF03D082
:1060D00003015551275E26506B2627506C226B50CA
:1060E0000001C65D6C50C7596C50C719D8B0800A02
:1060F00004E6C7C06CF0C6C06BF06CAE02D06C6A30
:106100006B6A800E016E19EC00F01D0EF76E860EA4
:10611000F66E3BEC01F0800E016E030E076E6CC054
:1061200022F06BC021F055C31BF01C6A78EC02F022
:106130001B6E14C01CF06FEC00F0050E43EC01F078
:106140003BEC43F0DAEF36F0040E965DD8A44DD068
:10615000975103015503F3CF26F0F4CF27F055AF45
:1061600001D0275E000197AF03D003015551275E90
:1061700026506D2627506E226D500001C85D6E506E
:10618000C9596E50C919D8B0800A07E6B051030149
:106190005503F4CF6EF0F3CF6DF000016EAE02D078
:1061A0006E6A6D6A800E016E19EC00F01D0EF76EBE
:1061B000980EF66E3BEC01F0800E016E030E076E3A
:1061C0006EC022F06DC021F055C31BF01C6A78EC44
:1061D00002F01B6E14C01CF06FEC00F0050E43ECD7
:1061E00001F03BEC43F0DAEF36F0050E965DD8A4F3
:1061F00049D0975103015503F3CF26F0F4CF27F090
:1062000055AF01D0275E000197AF03D00301555170
:10621000275E265075262750762275500001CE5DE8
:106220007650CF597650CF19D8B0800A04E6CFC047
:1062300076F0CEC075F076AE02D0766A756A800EC2
:10624000016E19EC00F01D0EF76EAA0EF66E3BEC17
:1062500001F0800E016E030E076E76C022F075C04D
:1062600021F055C31BF01C6A78EC02F01B6E14C0C1
:106270001CF06AEC00F0050E43EC01F03BEC43F03F
:10628000DAEF36F0060E965DD8A449D09751030197
:106290005503F3CF26F0F4CF27F055AF01D0275E9A
:1062A000000197AF03D003015551275E2650772692
:1062B0002750782277500001D05D7850D15978501E
:1062C000D119D8B0800A04E6D1C078F0D0C077F0F8
:1062D00078AE02D0786A776A800E016E19EC00F011
:1062E0001D0EF76EBC0EF66E3BEC01F0800E016EDB
:1062F000030E076E78C022F077C021F055C31BF063
:106300001C6A78EC02F01B6E14C01CF06AEC00F002
:10631000050E43EC01F03BEC43F0DAEF36F0070EEC
:10632000965DD8A4AFD0975103015503F3CF26F063
:10633000F4CF27F055AF01D0275E000197AF03D00F
:1063400003015551275E2650792627507A220001F5
:106350009A51E8B63FD0C651795CC7517A587A5005
:10636000C719D8B0800A04E6C7C07AF0C6C079F071
:1063700003015551A40DF3CF0BF0F4CF0CF00D6ACF
:106380000E6A5551010DF3500C26F4500D22000EEB
:106390000E2279C013F07AC014F0000E14BEFF0E66
:1063A000156E166E13500B5C14500C5815500D588A
:1063B00016500E580E501618D8B0800A000108E684
:1063C00003015551A40DF3CF79F0F4CF7AF07A267A
:1063D000000135D0C451795CC5517A587A50C5193D
:1063E000D8B0800A04E6C5C07AF0C4C079F00301D1
:1063F0005551F00DF3CF0BF0F4CF0CF00D6A0E6A8F
:1064000079C013F07AC014F0000E14BEFF0E156EA2
:10641000166E13500B5C14500C5815500D58165036
:106420000E580E501618D8B0800A000107E6030176
:106430005551F00DF3CF79F0F4CF7AF00001800ED2
:10644000016E19EC00F01D0EF76ECE0EF66E3BECF1
:1064500001F0800E016E030E076E7AC022F079C043
:1064600021F055C31BF01C6A78EC02F01B6E14C0BF
:106470001CF06FEC00F0050E43EC01F03BEC43F038
:10648000DAEF36F0080E965D23E197517B247B6EA0
:10649000000E97BFFF0E7C207C6E800E016E19EC03
:1064A00000F01D0EF76EE00EF66E3BEC01F0800E74
:1064B000016E030E076E7CC01CF07BC01BF06FECFE
:1064C00000F0050E43EC01F03BEC43F0DAEF36F060
:1064D000090E965D4DE19751E8BE03D0975301E058
:1064E000458A9751E8AE01D0459A800E016E19ECAD
:1064F00000F01D0EF76EF20EF66E3BEC01F045AAB1
:106500000AD04C0E43EC01F0430E43EC01F0440E74
:1065100043EC01F009D04C0E43EC01F0450E43EC86
:1065200001F0440E43EC01F0200E43EC01F0000EAC
:1065300043EC01F0200E43EC01F04D0E43EC01F072
:10654000200E43EC01F0010E43EC01F0200E43EC71
:1065500001F043EC01F043EC01F0040E43EC01F0D8
:106560001E0EF76E040EF66E3BEC01F0DAEF36F01D
:106570000A0E965D2CE19751E8BE03D0975301E0D7
:1065800043949751E8AE01D04384800E016E19EC1C
:1065900000F01E0EF76E100EF66E3BEC01F043A4F9
:1065A00009D04F0E43EC01F0460E43EC01F043ECF2
:1065B00001F009D0200E43EC01F04F0E43EC01F046
:1065C0004E0E43EC01F072EC43F0DAEF36F00B0EB6
:1065D000965D41E19751E8BE03D0975301E0438AAD
:1065E0009751E8AE01D0439A800E016E19EC00F08D
:1065F0001E0EF76E220EF66E3BEC01F043AA04D09D
:10660000420E43EC01F003D0410E43EC01F0200EAA
:1066100043EC01F0000E43EC01F0200E43EC01F0DE
:106620004D0E43EC01F0200E43EC01F0010E43EC63
:1066300001F0200E43EC01F043EC01F043EC01F0DB
:10664000040E43EC01F01E0EF76E360EF66E3BECB8
:1066500001F0DAEF36F00C0E965DD8A44CD09751CD
:10666000E8BE04D0975302E0B40EB06F9751E8AE85
:1066700002D05A0EB06FB05103015503F4CFC9F0E8
:10668000F3CFC8F0800E016E19EC00F01E0EF76E0D
:10669000420EF66E3BEC01F0800E016E030E076EAB
:1066A0000001B0516DEC00F0050E43EC01F0200E3E
:1066B00043EC01F0000E43EC01F0200E43EC01F03E
:1066C0004D0E43EC01F0200E43EC01F0010E43ECC3
:1066D00001F0200E43EC01F043EC01F043EC01F03B
:1066E000040E43EC01F01E0EF76E540EF66E3BECFA
:1066F00001F0DAEF36F00D0E965D47E19751E8BEF6
:1067000003D0975301E043869751E8AE01D04396FA
:10671000800E016E19EC00F01E0EF76E600EF66E24
:106720003BEC01F043B607D01E0EF76E700EF66E0E
:106730003BEC01F006D01E0EF76E780EF66E3BECC9
:1067400001F0200E43EC01F0000E43EC01F0200EAE
:1067500043EC01F04D0E43EC01F0200E43EC01F050
:10676000010E43EC01F0200E43EC01F043EC01F08C
:1067700043EC01F0040E43EC01F01E0EF76E800EA8
:10678000F66E3BEC01F0DAEF36F00E0E965D48E166
:106790009751E8BE04D0975302E04388438C975149
:1067A000E8AE02D04398438C800E016E19EC00F0E5
:1067B0001E0EF76E8C0EF66E3BEC01F043BC07D05C
:1067C0001E0EF76E960EF66E3BEC01F00FD043B83E
:1067D00007D01E0EF76EA20EF66E3BEC01F006D04F
:1067E0001E0EF76EAE0EF66E3BEC01F0200E43EC83
:1067F00001F0000E43EC01F0200E43EC01F04D0ED1
:1068000043EC01F0200E43EC01F0010E43EC01F0EB
:106810001E0EF76EBA0EF66E3BEC01F0DAEF36F0B4
:106820000F0E965DD8A451D09751E8AE11D0030E4B
:10683000895D0AE303E1E90E885D06E30A0E0001C3
:10684000885F000E895B04D0030E896FE80E886FA5
:106850009751E8BE11D097530FE0270E895D100EB7
:10686000D8B4885D05E20A0E8827000E892304D07B
:10687000270E896F100E886F800E016E19EC00F0E4
:106880001E0EF76ECA0EF66E3BEC01F0270E895D08
:10689000100ED8B4885D03E2200E43EC01F0800EA8
:1068A000016E076A89C01CF088C01BF06FEC00F015
:1068B000200E43EC01F0480E43EC01F07A0E43EC5D
:1068C00001F03BEC43F0DAEF36F0100E965D2AE172
:1068D000800E016E19EC00F01E0EF76ED80EF66EEB
:1068E0003BEC01F08EC329F08DC328F08CC327F058
:1068F0008BC326F0010EA7EC00F0200E43EC01F054
:1069000043EC01F043EC01F043EC01F043EC01F007
:10691000800E016E160E066E020E1C6E120E2BEC11
:1069200001F048D2110E965DD8A45BD09751E8BE15
:1069300011D097530FE0040E7D5C02E1020E7D6ED4
:106940000A0E7D5C02E1040E7D6E140E7D5C02E198
:106950000A0E7D6E9751E8AE0FD00A0E7D5C02E103
:10696000140E7D6E040E7D5C02E10A0E7D6E020E39
:106970007D5C02E1040E7D6E800E016E19EC00F06C
:106980001E0EF76EE60EF66E3BEC01F0140E7D5C0B
:1069900007E11E0EF76EF20EF66E3BEC01F01AD018
:1069A0000A0E7D5C07E11E0EF76EFC0EF66E3BECE8
:1069B00001F010D0040E7D5C07E11F0EF76E060E8D
:1069C000F66E3BEC01F006D01F0EF76E100EF66E61
:1069D0003BEC01F03BEC43F00301110E5C6F000156
:1069E000E9D1120E965D29E10301010EA06F81C06D
:1069F000A4F380C0A3F37FC0A2F37EC0A1F3000183
:106A000088EC45F0A8C381F0A7C380F0A6C37FF04F
:106A1000A5C37EF00301140E546F110E5C5D0001DE
:106A200003E1130E966F02D0110E966F0301120E42
:106A30005C6F000193EF2DF0BDD1130E965D29E13F
:106A40000301020EA06F85C0A4F384C0A3F383C02A
:106A5000A2F382C0A1F3000188EC45F0A8C385F041
:106A6000A7C384F0A6C383F0A5C382F00301140E6C
:106A7000546F120E5C5D000103E1140E966F02D09C
:106A8000120E966F0301130E5C6F000193EF2DF051
:106A900091D1140E965D31E197518625866F000ED7
:106AA00097BFFF0E8721876F8751E8AE02D0876BB3
:106AB000866B800E016E19EC00F01F0EF76E1A0E39
:106AC000F66E3BEC01F0800E016E040E076E87C07F
:106AD0001CF086C01BF06FEC00F0200E43EC01F0C0
:106AE0006D0E43EC01F0200E43EC01F03BEC43F063
:106AF0000301140E5C6F00015DD1150E965D2BE154
:106B00009751E8AE01D042989751E8BE03D0975311
:106B100001E04288800E016E19EC00F01F0EF76E46
:106B2000280EF66E3BEC01F042B809D04F0E43EC54
:106B300001F0460E43EC01F043EC01F009D0200EC9
:106B400043EC01F04F0E43EC01F04E0E43EC01F02C
:106B500072EC43F02FD1160E965D2BE19751E8AE03
:106B600001D0429A9751E8BE03D0975301E0428A80
:106B7000800E016E19EC00F01F0EF76E3A0EF66EE5
:106B80003BEC01F042BA09D04F0E43EC01F0460E47
:106B900043EC01F043EC01F009D0200E43EC01F08E
:106BA0004F0E43EC01F04E0E43EC01F072EC43F05B
:106BB00001D1170E965DD8A468D09751E8AE20D0C9
:106BC0008B51250A800ED8B48A1904E1120E8B6FFE
:106BD000C00E8A6F8B514B0A8A1104E1250E8B6F10
:106BE000800E8A6F8B51960A8A1103E14B0E8B6FD0
:106BF0008A6B8B51E10A8A1103E1960E8B6F8A6BC7
:106C00009751E8BE23D0975321E08B51960A8A1101
:106C100003E1E10E8B6F8A6B8B514B0A8A1103E102
:106C2000960E8B6F8A6B8B51250A800ED8B48A1909
:106C300003E14B0E8B6F8A6B8B51120AC00ED8B4D6
:106C40008A1904E1250E8B6F800E8A6F800E016E0B
:106C500019EC00F01F0EF76E4C0EF66E3BEC01F0D7
:106C6000270E8B5D100ED8B48A5D03E2200E43EC34
:106C700001F0800E016E076A8BC01CF08AC01BF009
:106C80006FEC00F03BEC43F095D0180E965D2BE1D5
:106C90009751E8BE03D0975301E043829751E8AE85
:106CA00001D04392800E016E19EC00F01F0EF76EBA
:106CB0005C0EF66E3BEC01F043A20AD0200E43ECD2
:106CC00001F04F0E43EC01F04E0E43EC01F008D002
:106CD0004F0E43EC01F0460E43EC01F043EC01F0A3
:106CE00072EC43F067D0190E965D2BE19751E8AE38
:106CF00001D044909751E8BE03D0975301E04480FF
:106D0000800E016E19EC00F01F0EF76E6E0EF66E1F
:106D10003BEC01F044B009D04F0E43EC01F0460EBD
:106D200043EC01F043EC01F009D0200E43EC01F0FC
:106D30004F0E43EC01F04E0E43EC01F072EC43F0C9
:106D400039D01A0E965D36E19751E8AE01D089D858
:106D50009751E8BE03D0975301E02AD9800E016E07
:106D600019EC00F01F0EF76E800EF66E3BEC01F092
:106D7000200E43EC01F0000E43EC01F0200E43EC3A
:106D800001F04D0E43EC01F0200E43EC01F0010E3A
:106D900043EC01F0200E43EC01F043EC01F043EC36
:106DA00001F0040E43EC01F01F0EF76E960EF66E26
:106DB0003BEC01F0976B010E80BC000E3B6E010EA8
:106DC00080BE000E3B1203E06AEC40F0F4D7BB6BD0
:106DD000BA6B010E82B4000E3B6E010E82B6000E3D
:106DE0003B1211E0030156510001BA27000EBB23EC
:106DF000BA51985DBB51995906E3010E14EC02F0AB
:106E00006AEC40F0E6D7995303E1330E985D05E351
:106E1000190E0001985F000E995B000E82B4010EFE
:106E20003B6E000E82B6010E3B16000E80BE010EB8
:106E30003B16000E80BC010E3B16000E82B2010E06
:106E40003B160BE0010E996FF40E986F6AEC40F060
:106E500003015453000101E0E0D793EF2DF0429C71
:106E60001200448E800E016E19EC00F01F0EF76EBA
:106E7000A20EF66E3BEC01F0800E016E940E19EC42
:106E800000F01F0EF76EB80EF66E3BEC01F080AE10
:106E9000FED7936B926B4590458293988A88070E34
:106EA000935DD00ED8B4925D33E24B50C15D06E1E4
:106EB0004A50C05D03E1924B932B06D04BC0C1F00A
:106EC0004AC0C0F0936B926B800E016E940E19EC69
:106ED00000F0030E076E4BC022F04AC021F055C3EC
:106EE0001BF01C6A78EC02F01B6E14C01CF06AECFC
:106EF00000F06AEC40F082B20AD093988A98449EDF
:106F00000301516B429E140E546F00011200C7D74B
:106F100093988A984B6A4A6A800E016E940E19EC17
:106F200000F01F0EF76EC20EF66E3BEC01F0449EB1
:106F30004592458093968A866F504A5C0B6E7050DE
:106F40004B580C6E0CAE2CD06F504A5C266E7050B5
:106F50004B58276E27C022F026C021F055C31BF0E6
:106F60001C6A78EC02F08C6F14C08DF0800E016EFC
:106F7000940E19EC00F0030E076E8DC01CF08CC04F
:106F80001BF06AEC00F06AEC40F0010E82B2000ED9
:106F90003B6E000E42BE010E3B1201E001D0CCD789
:106FA00093968A960301516B140E546F00011200E0
:106FB000448E800E016E19EC00F01F0EF76EA20ECB
:106FC000F66E3BEC01F0800E016E940E19EC00F0B1
:106FD0001F0EF76EB80EF66E3BEC01F080ACFED7DC
:106FE000936B926B4DC0C3F04CC0C2F04594458684
:106FF000939C8A8C070E935DD00ED8B4925D31E2DB
:107000004D50C35D06E14C50C25D03E1924B932BA2
:1070100006D04DC0C3F04CC0C2F0936B926B800E93
:10702000016E940E19EC00F0030E076E4DC022F0B5
:107030004CC021F055C31BF01C6A78EC02F01B6EAB
:1070400014C01CF06AEC00F06AEC40F082B208D088
:10705000449E0301526B4390140E546F00011200C2
:10706000C9D7939C8A9C4D6A4C6A800E016E940E1F
:1070700019EC00F01F0EF76EC20EF66E3BEC01F03D
:10708000449E45964584939A8A8A71504C5C0B6E57
:1070900072504D580C6E0CAE2CD071504C5C266E5C
:1070A00072504D58276E27C022F026C021F055C3DC
:1070B0001BF01C6A78EC02F08C6F14C08DF0800E0F
:1070C000016E940E19EC00F0030E076E8DC01CF0DB
:1070D0008CC01BF06AEC00F06AEC40F0010E82B24A
:1070E000000E3B6E000E43B0010E3B1201E001D0DA
:1070F000CCD7939A8A9A0301526B140E546F0001F5
:10710000120002EE28F0E9CFDEFFEACFDEFF030136
:107110009F6B00014BEC45F01FEEE9F016EC03F01D
:1071200013EEC4F0500EE75204E0E6CFEEFFE82E77
:10713000FAD7EF6A01EEB1F012EE28F0030E37EC49
:1071400003F0EF6A1F0EF76ECA0EF66E01EEB1F095
:1071500055EC03F03B6E000E42B0010E3B12000EE8
:1071600042B2010E3B1204E000EEF6F0EF6A1200AC
:10717000010EA56FA26B00EEF6F0A551EB500B6E61
:107180002A0E0B5C08E000EEF6F0A551EB500B6EFA
:10719000A21BA52BF0D7A52B00EEF6F0A551EB50C6
:1071A000186EFE0EF66E1F0EF76EF86A1768172A35
:1071B00017500F0806E30900F550185CF8E117C0F6
:1071C000A3F0A339F00BA46FA52B00EEF6F0A551A8
:1071D000EB50186E0E0EF66E200EF76EF86A1768FA
:1071E000172A17500F0806E30900F550185CF8E15C
:1071F00017C0A3F0A451A327A251A35D01E0120080
:1072000002EE28F0E9CFDEFFEACFDEFF0301020E37
:107210009F6F00014BEC45F01FEEE9F016EC03F018
:1072200013EEC4F0500EE75204E0E6CFEEFFE82E76
:10723000FAD7EF6A02012C510B6E2E0E0B5C000187
:1072400001E0120001EEB1F012EE28F0020EE6CFDE
:10725000EEFFE82EFCD7EF6A01EEB1F020EC00F073
:107260000301236F01EEB1F012EE28F0030EF36E6E
:10727000020E2EEC03F0EF6A01EEB1F020EC00F00C
:107280001EC035F01DC034F01CC033F01BC032F0FE
:1072900013EC09F035C027F334C026F333C025F3CF
:1072A00032C024F3010E03012353D8A4000E3B6E19
:1072B000356A346A336A326A27C339F026C338F034
:1072C00025C337F024C336F0ABEC06F03B160001C3
:1072D00001E0458CB40E0301235D010ED8A4000E1D
:1072E0003B6E356A346A336A326A27C339F026C383
:1072F00038F025C337F024C336F0ABEC06F03B166C
:10730000000101E0458C01EEB1F012EE28F0060E0E
:10731000F36E020E2EEC03F0EF6A01EEB1F020ECFA
:1073200000F01EC035F01DC034F01CC033F01BC08F
:1073300032F013EC09F035C06CF334C06BF333C09A
:107340006AF332C069F3396A386A480E376E850EBF
:10735000366E6CC335F06BC334F06AC333F069C367
:1073600032F002EC08F035C029F034C028F033C008
:1073700027F032C026F027C339F026C338F025C3E2
:1073800037F024C336F029C035F028C034F027C0C8
:1073900033F026C032F074EC07F035C027F334C068
:1073A00026F333C025F332C024F3396A386A700EED
:1073B000376E840E366E27C335F026C334F025C3EE
:1073C00033F024C332F002EC08F035C029F034C0A9
:1073D00028F033C027F032C026F0030123510FEC10
:1073E00009F029C039F028C038F027C037F026C08E
:1073F00036F074EC07F035C02BF334C02AF333C0F9
:1074000029F332C028F3356A346A340E336E850EA0
:10741000326E2BC339F02AC338F029C337F028C3A2
:1074200036F0F0EC06F00108000101E0120002EE77
:1074300028F0E9CFDEFFEACFDEFF0301030E9F6FE6
:1074400000014BEC45F01FEEE9F016EC03F013EEF3
:10745000C4F0500EE75204E0E6CFEEFFE82EFAD774
:10746000EF6A02EE28F0EECFF3FFEFCFF4FFF35018
:10747000530AF41002E10301297F000102EE28F013
:10748000E9CFDEFFEACFDEFF0301040E9F6F0001AC
:107490004BEC45F01FEEE9F016EC03F013EEC4F0F0
:1074A000500EE75204E0E6CFEEFFE82EFAD7EF6A7F
:1074B00002012D510B6E2E0E0B5C000101E012003B
:1074C00001EEB1F012EE28F0030EE6CFEEFFE82E4B
:1074D000FCD7EF6A01EEB1F020EC00F00301236F5E
:1074E00001EEB1F012EE28F0040EF36E020E2EEC57
:1074F00003F0EF6A01EEB1F020EC00F01EC035F0B1
:107500001DC034F01CC033F01BC032F013EC09F086
:1075100035C027F334C026F333C025F332C024F33B
:10752000010E03012353D8A4000E3B6E356A346A62
:10753000336A326A27C339F026C338F025C337F0DF
:1075400024C336F0ABEC06F03B16000E45BC010E32
:107550003B16000104E000EEF6F0EF6A120001EEC7
:10756000B1F012EE28F0070EF36E020E2EEC03F0CF
:10757000EF6A01EEB1F020EC00F01EC035F01DC046
:1075800034F01CC033F01BC032F013EC09F035C0EE
:107590006CF334C06BF333C06AF332C069F3396AF9
:1075A000386A480E376E850E366E6CC335F06BC385
:1075B00034F06AC333F069C332F002EC08F035C02E
:1075C00029F034C028F033C027F032C026F027C39A
:1075D00039F026C338F025C337F024C336F029C06C
:1075E00035F028C034F027C033F026C032F074ECF8
:1075F00007F035C027F334C026F333C025F332C07B
:1076000024F3396A386A700E376E840E366E27C3DB
:1076100035F026C334F025C333F024C332F002EC36
:1076200008F035C029F034C028F033C027F032C04C
:1076300026F0030123510FEC09F029C039F028C0CE
:1076400038F027C037F026C036F074EC07F035C0AC
:107650002FF334C02EF333C02DF332C02CF3356A30
:10766000346A340E336E860E326E2FC339F02EC359
:1076700038F02DC337F02CC336F0B8EC06F0010813
:10768000000101E0120002EE28F0E9CFDEFFEACFB0
:10769000DEFF0301050E9F6F00014BEC45F01FEE6E
:1076A000E9F016EC03F013EEC4F0500EE75204E0DC
:1076B000E6CFEEFFE82EFAD7EF6A02EE28F0EECF23
:1076C000F3FFEFCFF4FFF350570AF41002E1030188
:1076D0002D7F000102EE28F0E9CFDEFFEACFDEFFCA
:1076E0000301090E9F6F00014BEC45F01FEEE9F01E
:1076F00016EC03F013EEC4F0500EE75204E0E6CFB0
:10770000EEFFE82EFAD7EF6A02EE28F020EC00F048
:107710000301386F1CC039F301EEB1F012EE28F00E
:10772000010E37EC03F0EF6A0101B1510B6E350E1B
:107730000B5C000103E30301384B392B9C0E030162
:10774000395D000108E305E1410E0301385D0001E8
:1077500002E300011200D00E356E0F0E346E490E9A
:10776000336E800E326E2BC339F02AC338F029C332
:1077700037F028C336F068EC08F035C029F034C083
:1077800028F033C027F032C026F0396A386A340E48
:10779000376E860E366E29C035F028C034F027C00B
:1077A00033F026C032F002EC08F035C06CF334C080
:1077B0006BF333C06AF332C069F36CC335F06BC34B
:1077C00034F06AC333F069C332F091EC04F035C091
:1077D000AFF034C0AEF033C0ADF032C0ACF02FC368
:1077E00029F02EC328F02DC327F02CC326F029C082
:1077F00035F028C034F027C033F026C032F041C342
:1078000039F040C338F03FC337F03EC336F072EC76
:1078100007F035C029F034C028F033C027F032C05B
:1078200026F029C039F028C038F027C037F026C02C
:1078300036F0AFC035F0AEC034F0ADC033F0ACC000
:1078400032F068EC08F035C029F034C028F033C0BD
:1078500027F032C026F09A0E356E990E346E5E0E09
:10786000336E850E326E29C039F028C038F027C03B
:1078700037F026C036F068EC08F035C04BF334C062
:107880004AF333C049F332C048F32BC335F02AC35F
:1078900034F029C333F028C332F03DC339F03CC380
:1078A00038F03BC337F03AC336F072EC07F035C01E
:1078B00029F034C028F033C027F032C026F09A0EE9
:1078C000356E990E346E5E0E336E850E326E29C0A3
:1078D00039F028C038F027C037F026C036F068EC01
:1078E00008F035C047F334C046F333C045F332C027
:1078F00044F347C339F046C338F045C337F044C3B7
:1079000036F047C335F046C334F045C333F044C3C3
:1079100032F068EC08F0B6EC08F003016D6F33C08C
:107920006EF334C06FF335C070F34BC339F04AC304
:1079300038F049C337F048C336F04BC335F04AC37B
:1079400034F049C333F048C332F068EC08F0B6ECC9
:1079500008F00301716F33C072F334C073F335C0A4
:1079600074F371516D255D6F72516E215E6F7351AD
:107970006F215F6F74517021606F60C335F05FC31A
:1079800034F05EC333F05DC332F015EC09F000EC67
:1079900006F035C080F334C07FF333C07EF332C0CD
:1079A0007DF3396A386A7A0E376E880E366E43C3B5
:1079B00033F042C332F009EC09F002EC08F035C0B4
:1079C00029F034C028F033C027F032C026F0356AE1
:1079D000500E346E470E336E8B0E326E29C039F066
:1079E00028C038F027C037F026C036F074EC07F016
:1079F00035C07CF334C07BF333C07AF332C079F303
:107A00007CC339F07BC338F07AC337F079C336F0E2
:107A10007CC335F07BC334F07AC333F079C332F0E2
:107A200068EC08F0B6EC08F003016D6F33C06EF33C
:107A300034C06FF335C070F380C339F07FC338F0C2
:107A40007EC337F07DC336F080C335F07FC334F09A
:107A50007EC333F07DC332F068EC08F0B6EC08F07A
:107A60000301716F33C072F334C073F335C074F324
:107A700071516D255D6F72516E215E6F73516F2173
:107A80005F6F74517021606F60C335F05FC334F075
:107A90005EC333F05DC332F015EC09F000EC06F084
:107AA00035C0AFF034C0AEF033C0ADF032C0ACF092
:107AB000AFC029F0AEC028F0ADC027F0ACC026F0B2
:107AC00029C035F028C034F027C033F026C032F08A
:107AD0007CC339F07BC338F07AC337F079C336F012
:107AE00072EC07F035C029F034C028F033C027F01D
:107AF00032C026F0356A346A7A0E336E880E326EE2
:107B000029C039F028C038F027C037F026C036F039
:107B100068EC08F035C029F034C028F033C027F0F5
:107B200032C026F043C333F042C332F009EC09F00F
:107B300029C039F028C038F027C037F026C036F009
:107B400074EC07F0B6EC08F003016D6F33C06EF310
:107B500034C06FF335C070F370530001D8A49FD0C8
:107B600003016F530001D8A49AD003016E51395D0F
:107B70000001D8A094D006E1030138516D5D0001E9
:107B8000D8B08DD003016D51385D716F6E51395988
:107B9000726F000E6F55736F000E7055746F80C357
:107BA00039F07FC338F07EC337F07DC336F074C33D
:107BB00035F073C334F072C333F071C332F013EC99
:107BC00009F002EC08F035C029F034C028F033C0C9
:107BD00027F032C026F0396A386A7A0E376E880E7E
:107BE000366E29C035F028C034F027C033F026C0E7
:107BF00032F002EC08F035C0AFF034C0AEF033C064
:107C0000ADF032C0ACF0AFC035F0AEC034F0ADC0B6
:107C100033F0ACC032F05FEC03F035C06CF334C02D
:107C20006BF333C06AF332C069F36CC337F36BC3D1
:107C300036F36AC335F369C334F3356A346A340EF4
:107C4000336E860E326E6CC339F06BC338F06AC384
:107C500037F069C336F068EC08F035C029F034C05D
:107C600028F033C027F032C026F0D00E396E0F0E48
:107C7000386E490E376E800E366E29C035F028C03A
:107C800034F027C033F026C032F002EC08F068EC84
:107C900007F00301816F33C082F3000103D00301B9
:107CA000826B816B0301825304E15B0E815D0001F5
:107CB00004E3496A486A0001120003015551810337
:107CC000F3CF48F0F4CF49F08203F3504926000186
:107CD00049AE03D0496A486A120049C033F048C02F
:107CE00032F009EC09F035C037F334C036F333C055
:107CF00035F332C034F34850BE5D136E4950BF595E
:107D0000146E03EC03F00B6E14C00CF0030155511C
:107D1000050DF3CF0FF0F4CF10F0116A126A125272
:107D2000000114E1115212E110500C5C0FE303E169
:107D30000B500F5C0BE20001A82B030EA85D05E3BE
:107D400049C0BFF048C0BEF0A86B01D0A86B4BC3C0
:107D500035F04AC334F049C333F048C332F047C367
:107D600039F046C338F045C337F044C336F002EC6F
:107D700008F035C0AFF034C0AEF033C0ADF032C063
:107D8000ACF0AFC035F0AEC034F0ADC033F0ACC035
:107D900032F05FEC03F035C06CF334C06BF333C0EA
:107DA0006AF332C069F3356A346A340E336E860E74
:107DB000326E6CC339F06BC338F06AC337F069C3F5
:107DC00036F068EC08F035C029F034C028F033C034
:107DD00027F032C026F0D00E396E0F0E386E490EE5
:107DE000376E800E366E29C035F028C034F027C0BB
:107DF00033F026C032F002EC08F035C06CF334C02A
:107E00006BF333C06AF332C069F36CC333F36BC3F3
:107E100032F36AC331F369C330F36CC335F06BC31B
:107E200034F06AC333F069C332F068EC07F0030141
:107E3000816F33C082F347C335F046C334F045C386
:107E400033F044C332F0396A386A376A366AF0EC84
:107E500006F03B6E4BC335F04AC334F049C333F0F0
:107E600048C332F0396A386A376A366A2CEC07F050
:107E70003B1600011DE0680E03018127010E8223DD
:107E8000356A346A340E336E870E326E33C339F07E
:107E900032C338F031C337F030C336F074EC07F03A
:107EA00035C033F334C032F333C031F332C030F372
:107EB000030145510001E8AE1DD0B40E0301812736
:107EC000000E8223356A346A340E336E860E326EAB
:107ED00033C339F032C338F031C337F030C336F032
:107EE00074EC07F035C033F334C032F333C031F3F0
:107EF00032C030F3000182C347F081C346F0030172
:107F000081510001BC5D136E030182510001BD5916
:107F1000146E03EC03F00B6E14C00CF00C5203E172
:107F2000060E0B5C0BE30001A72B030EA75D05E318
:107F300082C3BDF081C3BCF0A76B01D0A76B00EE7C
:107F4000F6F0EF6AA75302E1000E01D0010E3B6E7E
:107F5000A85302E1000E01D0010E3B1201E0120015
:107F600082C3BDF081C3BCF049C0BFF048C0BEF0C1
:107F70001E0E03015B5D000101E212000301555179
:107F80008103F3CF46F0F4CF47F08203F350472646
:107F900047C09AF346C099F300015EEC44F09CC3DD
:107FA0005FF09BC35EF043BE43D06F504A5C0B6EE4
:107FB00070504B580C6E70BEFF0E000E0D6A4BBE1B
:107FC0000D6870BEFF0E0D5A0E6A0DBE0E680B5086
:107FD0005E180BE10C505F1808E10D505FBE0D28D4
:107FE00004E10E505FBE0E2801E042800001715096
:107FF0004C5C0B6E72504D580C6E72BEFF0E000E34
:108000000D6A4DBE0D6872BEFF0E0D5A0E6A0DBE92
:108010000E680B5048180BE10C50491808E10D5040
:1080200049BE0D2804E10E5049BE0E2801E04282EF
:1080300003015B6B000E42B0010E3B6E000E42B2BC
:10804000010E3B12000101E001D812009A51E8BA7A
:1080500001D01200000E81B6010E3B6E000E81B8F9
:10806000010E3B12000E81BA010E3B12000E81BCC4
:10807000010E3B1201E012009A51E8A824D0610ED3
:10808000146EA80E136E84C318F083C317F061EC4E
:1080900002F00A6EA06BA0510A5C13E3939E8A8ED5
:1080A00084C314F00301835122EC02F0939E8A9E54
:1080B00084C314F00301835122EC02F00001A02BD1
:1080C000EAE3938E06D0939E8A8E320E14EC02F071
:1080D000938E1200E86A44B2010F81B00108D8A45F
:1080E000010E3B6EE86A44B4010F81B20108D8A4C6
:1080F000010E3B12D8B458D0020E14EC02F0E86A1C
:1081000044B2010F81B00108D8A4010E3B6EE86AA9
:1081100044B4010F81B20108D8A4010E3B12D8B4B7
:1081200043D0020E14EC02F0E86A44B2010F81B0B1
:10813000010819E0448281A0449245A002D04A4A35
:108140004B2A45A204D0010E4A5E000E4B5AE86A43
:1081500081B6010F81B8010804E193968A9693983D
:108160008A980301516B0001E86A44B4010F81B29F
:10817000010819E0448481A2449445A402D04C4AE9
:108180004D2A45A604D0010E4C5E000E4D5AE86AF9
:1081900081BC010F81BA010804E1939A8A9A939CE9
:1081A0008A9C0301526B00011200840E026E020EC3
:1081B000086E840E036E010E046E050E096ED45116
:1081C000136EEBEC01F0D551136EEBEC01F0D651D0
:1081D000136EEBEC01F0D751136EEBEC01F0D851BC
:1081E000136EEBEC01F0D951136EEBEC01F09694A9
:1081F0008D8496948D941200000100C031F401C06A
:1082000032F4A9CF33F4AACF34F4A6CF35F4A7CFF4
:1082100036F4A8CF37F4EACF38F4E9CF39F4E2CF17
:108220003AF4E1CF3BF413C03CF414C03DF41FC05A
:108230003EF420C03FF421C040F4F3CF41F43BC0F2
:1082400042F49EAA54D0AECFA9F0610EA95D000EF3
:10825000D8B0010E3B6E7B0EA95D02E3000E01D08B
:10826000010E3B1601E0A99B9A3103E3A951B7EC3B
:1082700001F09E9A0A0EA95D17E001EE47F0EE505C
:10828000FEE1ED52A9C0EEFFEF6A4E0E0301505D14
:10829000000104E20301502B000105D00301506BE3
:1082A00001EE47F0EF6A0001240EA95D08E101EE3E
:1082B00047F0EF6A01EE47F0A9C0EEFFEF6A0D0E3E
:1082C000A95D15E1448C0301506B0001D20EAB6F28
:1082D00000EEF6F011EE47F0500EE75204E0E6CF64
:1082E000EEFFE82EFAD7EF6A01EE47F0EF6AF0A250
:1082F0002AD00EEC00F093968A9693988A98939AD7
:108300008A9A939C8A9C95968C96AA6AA96A4A50E6
:10831000CFEC01F04B50CFEC01F0AA6A020EA96E2F
:108320004C50CFEC01F04D50CFEC01F0AA6A210E79
:10833000A96E03018951CFEC01F003018A51CFEC02
:1083400001F00001FED731C400F032C401F033C4A3
:10835000A9FF34C4AAFF35C4A6FF36C4A7FF37C49B
:10836000A8FF38C4EAFF39C4E9FF3AC4E2FF3BC4BE
:10837000E1FF3CC413F03DC414F03EC41FF03FC401
:1083800020F040C421F041C4F3FF42C43BF011008F
:10839000F29EE0CF43F43BC044F4D8CF45F4E8CF9D
:1083A00046F4F28E00019EA468D09E949F2B0F0E7F
:1083B0009F5DD8A062D09F6B000E45B8010E010AE8
:1083C000D8B44598D8A44588000E43B0010E3B6E42
:1083D000000E42BE010E3B120DE0AA2B0D0EAA5D4F
:1083E00009E34390429E0301516B526B0001AA6B5B
:1083F00042904292FA0E03015B5D000102E203012A
:108400005B2B03015453000102E0030154070001F8
:1084100044BE2BD0000E81B6010E3B6E000E81B81B
:10842000010E3B1202E00301512B0001000E81BA44
:10843000010E3B6E000E81BC010E3B1202E00301F7
:10844000522B050E0301515D000105E3428E939806
:108450008A9893968A96050E0301525D000105E302
:108460004380939A8A9A939C8A9CBE0E0301875DEF
:10847000000102E20301872B0001F29E43C4E0FFEA
:1084800044C43BF045C4D8FF46C4E8FFF28E100058
:10849000AA6A040EA96EE4EC01F0676EE4EC01F048
:1084A000686EAA6A060EA96EE4EC01F0696EE4EC4F
:1084B00001F06A6EAA6A080EA96EE4EC01F06F6E14
:1084C000E4EC01F0706EAA6A0A0EA96EE4EC01F009
:1084D000716EE4EC01F0726EAA6A0C0EA96EE4EC07
:1084E00001F0736EE4EC01F0746EAA6A0E0EA96ED0
:1084F000E4EC01F0666EAA6A0F0EA96EE4EC01F0DE
:108500009A6FAA6A100EA96EE4EC01F00301596F8C
:10851000AA6A110EA96EE4EC01F00301556FAA6A74
:10852000120EA96EE4EC01F003013A6FE4EC01F0E5
:1085300003013B6FE4EC01F003013C6FE4EC01F05C
:1085400003013D6FAA6A160EA96EE4EC01F0030167
:108550003E6FE4EC01F003013F6FE4EC01F0030136
:10856000406FE4EC01F00301416FAA6A1A0EA96E94
:10857000E4EC01F00301426FE4EC01F00301436F0E
:10858000AA6A1C0EA96EE4EC01F00301856FE4EC0D
:1085900001F00301866FC30E146E500E136E86C376
:1085A00018F085C317F061EC02F00301836F14C06B
:1085B00084F386510A0DF3CF86F385510A0DF3CF6C
:1085C00085F3F4508627020E555DD8A4010E3B6E4C
:1085D000040E555DD8A4010E3B160A0E555DD8A4B5
:1085E000010E3B16140E555DD8A4010E3B1600017A
:1085F00003E00301040E556F00014BC057F04AC061
:1086000056F04DC059F04CC058F003015551B40D0F
:10861000F3CFC4F0F4CFC5F05551680DF3CFC6F0D9
:10862000F4CFC7F00001C727665003015503F4CF0C
:10863000C9F0F3CFC8F055510A0DF3CFCAF0F4CF0B
:10864000CBF05551640DF3CFCCF0F4CFCDF05551B4
:108650001E0DF3CFD0F0F4CFD1F05551320DF3CF42
:10866000CEF0F4CFCFF055510F0DF3CFD2F0F4CFC1
:10867000D3F000011200200E43EC01F0000E43EC99
:1086800001F0200E43EC01F04D0E43EC01F0200E02
:1086900043EC01F0010E43EC01F0200E43EC01F03D
:1086A00043EC01F043EC01F0040E43EC01F0200E2A
:1086B00043EC01F043EC01F043EC01F043EC01F03A
:1086C000000E43EC01F0200E43EC01F0560E43EC9B
:1086D00001F0200E43EC01F0010E43EC01F0200EFE
:1086E00043EF01F0200E43EC01F0000E43EC01F0EB
:1086F000200E43EC01F04D0E43EC01F0200E43EC54
:1087000001F0010E43EC01F0200E43EC01F043ECCC
:1087100001F043EC01F0040E43EC01F01F0EF76E84
:10872000CE0EF66E3BEF01F0080EB86EAC98AC843E
:1087300003018851880DF3CF6DF3F4CF6EF36F6BA7
:10874000706B8851130DF3506E27F4506F23000E99
:108750007023B9C014F0B8C013F0186A640E176E15
:1087600061EC02F00001906F14C091F070C329F029
:108770006FC328F06EC327F06DC326F029C016F032
:1087800028C015F027C014F026C013F090C01BF0CD
:1087900091C01CF01D6A1E6A36EC02F016C029F06A
:1087A00015C028F014C027F013C026F02606000ECE
:1087B000275A285A295A28302730916F2630906F2F
:1087C00091C0B0FF90C0AFFF1200FFD7FFD7B76BCB
:1087D000B66BB7530CE1640EB65D09E2030E14EC00
:1087E00002F06AEC40F0B62B000EB723F2E3120061
:1087F000030155518F03F3CF46F0F4CF47F09003B8
:10880000F3504726428048500001C85D4950C9597D
:108810004950C919D8B0800A19E64850C45D486E5D
:108820004950C559496EC4514626C5514722C651C3
:10883000465CC75147584750C719D8B0800A06E769
:10884000C651465C466EC7514758476E47C09AF3BB
:1088500046C099F333D89CC35FF09BC35EF047C01A
:1088600092F346C091F31200030155519303F3CFE5
:1088700097F3F4CF98F39403F350982742829751DB
:108880000001C85D030198510001C95903019851C5
:108890000001C919D8B0800A0BE603019751000105
:1088A000C45D0301976F98510001C5590301986F8A
:1088B000000198C396F397C395F312009A51E8A666
:1088C00016D0C4510301995D9D6F0001C55103018C
:1088D0009A599E6F9E510001E8AE07D0C651030120
:1088E0009D270001C75103019E23000104D09AC3B4
:1088F0009EF399C39DF36F5003019D2770509E23F3
:1089000000019A35D8A0C2D074BE10D0120E745C8B
:108910000DE303E15D0E735C09E3AA6A0C0EA96E18
:10892000E4EC01F0736EE4EC01F0746E0001C651EA
:1089300003019D250B6E0001C75103019E210C6EA2
:1089400073500B5C74500C580C507418D8B0800ADB
:10895000000102E7000E01D0010E3B6E03015551EC
:108960000E0DF3CF26F0F4CF27F0286A2726000E4D
:10897000282255AF04D00E0E275E010E285A0001A2
:10898000296A28BE29066F5026240B6E70502720B6
:108990000C6E000E70BEFF0E28200D6E000E70BE15
:1089A000FF0E29200E6E4AC013F04BC014F0000ECB
:1089B00014BEFF0E156E166E13500B5C14500C583F
:1089C00015500D5816500E5816500E18D8B0800A73
:1089D00002E7000E01D0010E3B1607E0C65103016D
:1089E0009D270001C75103019E2300016F50CE2532
:1089F0000B6E7050CF210C6E000E0CBEFF0E0D6E74
:108A00000E6E4AC013F04BC014F0000E14BEFF0EE1
:108A1000156E166E0B50135C0C5014580D501558F3
:108A20000E5016580E501618D8B0800A02E7000EE5
:108A300001D0010E3B6EC65103019D5D0B6E00011E
:108A4000C75103019E590C6E000E55BFFF0E0C5C02
:108A500007E00C505519D8B0800A800B07E008D009
:108A600000010B500301555D000102E3000E01D02F
:108A7000010E3B16000109E0C65103019D5D9D6F8B
:108A80000001C75103019E599E6F00019EC39CF3D4
:108A90009DC39BF31200A66B03019F53000118E0D6
:108AA00000EEF6F0A651EB500B6E2C0E0B5CD8A42A
:108AB000010E3B6E500EA65D010ED8B0000E3B16A7
:108AC00002E0A62BEDD7A62B03019F070001E4D7F8
:108AD000A56B00EEF6F0A651EB500B6E2C0E0B5C66
:108AE00010E000EEF6F0A651EBCF0BF003EEC4F071
:108AF000A5510BC0EBFF4E0EA55D01E2A52BA62BE9
:108B0000E8D7F36A03EEC4F0A551F3CFEBFF1200F0
:108B10000301A0510FEC09F0396A386A340E376E40
:108B2000850E366E68EC08F035C0ACF334C0ABF39C
:108B300033C0AAF332C0A9F30301A0510E085A6F43
:108B40000001010E80BE000E3B6E010E80BC000EC7
:108B50003B12010E82B4000E3B12010E82B6000ED3
:108B60003B1201E0EDD782A297EF4AF05AC3BEF361
:108B7000A0C3BFF3A4C3C3F3A3C3C2F3A2C3C1F38F
:108B8000A1C3C0F385EC4BF082B4B9D10C0E030144
:108B90005A5D010ED8A4000E3B6E020EA05D010EC0
:108BA000D8A4000E3B16A4C335F0A3C334F0A2C36F
:108BB00033F0A1C332F0396A386A480E376E850E39
:108BC000366EB8EC06F03B16000118E0396A386AD8
:108BD000480E376E850E366EA4C335F0A3C334F04D
:108BE000A2C333F0A1C332F072EC07F035C0A4F396
:108BF00034C0A3F333C0A2F332C0A1F30D0E0301BE
:108C00005A5D010ED8A4000E3B6EA4C335F0A3C379
:108C100034F0A2C333F0A1C332F0396A386A200EAF
:108C2000376E820E366EB8EC06F03B16000118E087
:108C3000396A386A200E376E820E366EA4C335F05C
:108C4000A3C334F0A2C333F0A1C332F072EC07F037
:108C500035C0A4F334C0A3F333C0A2F332C0A1F3F0
:108C60000E0E03015A5D010ED8A4000E3B6EA4C384
:108C700035F0A3C334F0A2C333F0A1C332F0396A94
:108C8000386A376A7F0E366EB8EC06F03B16000184
:108C900017E0396A386A376A7F0E366EA4C335F03A
:108CA000A3C334F0A2C333F0A1C332F072EC07F0D7
:108CB00035C0A4F334C0A3F333C0A2F332C0A1F390
:108CC000100E03015A5D010ED8A4000E3B6EA4C322
:108CD00035F0A3C334F0A2C333F0A1C332F0CD0EFC
:108CE000396ECC0E386E4C0E376E7B0E366EB8EC8D
:108CF00006F03B1600011AE0CD0E396ECC0E386E30
:108D00004C0E376E7B0E366EA4C335F0A3C334F021
:108D1000A2C333F0A1C332F072EC07F035C0A4F364
:108D200034C0A3F333C0A2F332C0A1F3110E030188
:108D30005A5D010ED8A4000E3B6EA4C335F0A3C348
:108D400034F0A2C333F0A1C332F00A0E396ED70E4D
:108D5000386E230E376E780E366EB8EC06F03B1682
:108D600000011AE00A0E396ED70E386E230E376EE8
:108D7000780E366EA4C335F0A3C334F0A2C333F02B
:108D8000A1C332F072EC07F035C0A4F334C0A3F3F2
:108D900033C0A2F332C0A1F3120E03015A5D010EDB
:108DA000D8A4000E3B6EA4C335F0A3C334F0A2C315
:108DB00033F0A1C332F06F0E396E120E386E030E0F
:108DC000376E750E366EB8EC06F03B1600011AE0F1
:108DD0006F0E396E120E386E030E376E750E366ECC
:108DE000A4C335F0A3C334F0A2C333F0A1C332F05F
:108DF00072EC07F035C0A4F334C0A3F333C0A2F380
:108E000032C0A1F3130E03015A5D010ED8A4000E67
:108E10003B6EA4C335F0A3C334F0A2C333F0A1C3A7
:108E200032F0170E396EB70E386E510E376E710E66
:108E3000366EB8EC06F03B1600011AE0170E396EDC
:108E4000B70E386E510E376E710E366EA4C335F004
:108E5000A3C334F0A2C333F0A1C332F072EC07F025
:108E600035C0A4F334C0A3F333C0A2F332C0A1F3DE
:108E7000140E03015A5D010ED8A4000E3B6EA4C36C
:108E800035F0A3C334F0A2C333F0A1C332F0AC0E6B
:108E9000396EC50E386E270E376E6E0E366EB8EC14
:108EA00006F03B1600011AE0AC0E396EC50E386EA6
:108EB000270E376E6E0E366EA4C335F0A3C334F0A2
:108EC000A2C333F0A1C332F072EC07F035C0A4F3B3
:108ED00034C0A3F333C0A2F332C0A1F345985AC300
:108EE000BEF3A0C3BFF3A4C3C3F3A3C3C2F3A2C31F
:108EF000C1F3A1C3C0F385EC4BF082A4FED782B6C8
:108F000045EF4AF00C0E03015A5D010ED8A4000E85
:108F10003B6E020EA05D010ED8A4000E3B160001B0
:108F2000D8B44DD0396A386A480E376E850E366E21
:108F3000ACC335F0ABC334F0AAC333F0A9C332F0ED
:108F400072EC07F035C00EF034C00DF033C00CF0F9
:108F500032C00BF0A4C335F0A3C334F0A2C333F086
:108F6000A1C332F00EC039F00DC038F00CC037F09C
:108F70000BC036F0F0EC06F0010819E0356A346AEF
:108F8000480E336E850E326EA4C339F0A3C338F099
:108F9000A2C337F0A1C336F074EC07F035C0A4F3D8
:108FA00034C0A3F333C0A2F332C0A1F308D0ACC3E2
:108FB000A4F3ABC3A3F3AAC3A2F3A9C3A1F30D0EF9
:108FC00003015A5D0001D8A44DD0396A386A200ED9
:108FD000376E820E366EACC335F0ABC334F0AAC325
:108FE00033F0A9C332F072EC07F035C00EF034C094
:108FF0000DF033C00CF032C00BF0A4C335F0A3C3A6
:1090000034F0A2C333F0A1C332F00EC039F00DC06A
:1090100038F00CC037F00BC036F0F0EC06F0010869
:1090200019E0356A346A200E336E820E326EA4C3A4
:1090300039F0A3C338F0A2C337F0A1C336F074EC03
:1090400007F035C0A4F334C0A3F333C0A2F332C099
:10905000A1F308D0ACC3A4F3ABC3A3F3AAC3A2F398
:10906000A9C3A1F30E0E03015A5D0001D8A44BD091
:10907000396A386A376A7F0E366EACC335F0ABC3D7
:1090800034F0AAC333F0A9C332F072EC07F035C054
:109090000EF034C00DF033C00CF032C00BF0A4C39E
:1090A00035F0A3C334F0A2C333F0A1C332F00EC035
:1090B00039F00DC038F00CC037F00BC036F0F0ECD2
:1090C00006F0010818E0356A346A336A7F0E326EA2
:1090D000A4C339F0A3C338F0A2C337F0A1C336F05C
:1090E00074EC07F035C0A4F334C0A3F333C0A2F38B
:1090F00032C0A1F308D0ACC3A4F3ABC3A3F3AAC39B
:10910000A2F3A9C3A1F3100E03015A5D0001D8A474
:1091100051D0CD0E396ECC0E386E4C0E376E7B0EA4
:10912000366EACC335F0ABC334F0AAC333F0A9C379
:1091300032F072EC07F035C00EF034C00DF033C0E1
:109140000CF032C00BF0A4C335F0A3C334F0A2C3BB
:1091500033F0A1C332F00EC039F00DC038F00CC0AE
:1091600037F00BC036F0F0EC06F001081BE0CD0E36
:10917000356ECC0E346E4C0E336E7B0E326EA4C345
:1091800039F0A3C338F0A2C337F0A1C336F074ECB2
:1091900007F035C0A4F334C0A3F333C0A2F332C048
:1091A000A1F308D0ACC3A4F3ABC3A3F3AAC3A2F347
:1091B000A9C3A1F3110E03015A5D0001D8A451D037
:1091C0000A0E396ED70E386E230E376E780E366E55
:1091D000ACC335F0ABC334F0AAC333F0A9C332F04B
:1091E00072EC07F035C00EF034C00DF033C00CF057
:1091F00032C00BF0A4C335F0A3C334F0A2C333F0E4
:10920000A1C332F00EC039F00DC038F00CC037F0F9
:109210000BC036F0F0EC06F001081BE00A0E356ECC
:10922000D70E346E230E336E780E326EA4C339F02F
:10923000A3C338F0A2C337F0A1C336F074EC07F033
:1092400035C0A4F334C0A3F333C0A2F332C0A1F3FA
:1092500008D0ACC3A4F3ABC3A3F3AAC3A2F3A9C3BE
:10926000A1F3120E03015A5D0001D8A451D06F0E74
:10927000396E120E386E030E376E750E366EACC335
:1092800035F0ABC334F0AAC333F0A9C332F072ECAB
:1092900007F035C00EF034C00DF033C00CF032C012
:1092A0000BF0A4C335F0A3C334F0A2C333F0A1C3C1
:1092B00032F00EC039F00DC038F00CC037F00BC0E2
:1092C00036F0F0EC06F001081BE06F0E356E120E62
:1092D000346E030E336E750E326EA4C339F0A3C321
:1092E00038F0A2C337F0A1C336F074EC07F035C0F4
:1092F000A4F334C0A3F333C0A2F332C0A1F308D067
:10930000ACC3A4F3ABC3A3F3AAC3A2F3A9C3A1F351
:10931000130E03015A5D0001D8A451D0170E396E07
:10932000B70E386E510E376E710E366EACC335F017
:10933000ABC334F0AAC333F0A9C332F072EC07F028
:1093400035C00EF034C00DF033C00CF032C00BF05D
:10935000A4C335F0A3C334F0A2C333F0A1C332F0E9
:109360000EC039F00DC038F00CC037F00BC036F02D
:10937000F0EC06F001081BE0170E356EB70E346EE8
:10938000510E336E710E326EA4C339F0A3C338F0A0
:10939000A2C337F0A1C336F074EC07F035C0A4F3D4
:1093A00034C0A3F333C0A2F332C0A1F308D0ACC3DE
:1093B000A4F3ABC3A3F3AAC3A2F3A9C3A1F3140EEE
:1093C00003015A5D0001D8A451D0AC0E396EC50E10
:1093D000386E270E376E6E0E366EACC335F0ABC3EB
:1093E00034F0AAC333F0A9C332F072EC07F035C0F1
:1093F0000EF034C00DF033C00CF032C00BF0A4C33B
:1094000035F0A3C334F0A2C333F0A1C332F00EC0D1
:1094100039F00DC038F00CC037F00BC036F0F0EC6E
:1094200006F001081BE0AC0E356EC50E346E270E3B
:10943000336E6E0E326EA4C339F0A3C338F0A2C3EC
:1094400037F0A1C336F074EC07F035C0A4F334C094
:10945000A3F333C0A2F332C0A1F308D0ACC3A4F38A
:10946000ABC3A3F3AAC3A2F3A9C3A1F35AC3BEF328
:10947000A0C3BFF3A4C3C3F3A3C3C2F3A2C3C1F386
:10948000A1C3C0F342D982A6FED780BE2AD0030171
:109490005A07A0510D080B6E000ED8A0FF0F0C6EDE
:1094A0000C5204E15A510B5C000103E30301140E5A
:1094B0005A6F0F0E03015A5D000102E103015A07C2
:1094C000000145885AC3BEF3A0C3BFF3A4C3C3F3CE
:1094D000A3C3C2F3A2C3C1F3A1C3C0F316D980AE24
:1094E000FED780BC22D003015A2B150E5A5D000115
:1094F00004E30301A0510E085A6F0F0E03015A5DD9
:10950000000102E103015A2B000145885AC3BEF352
:10951000A0C3BFF3A4C3C3F3A3C3C2F3A2C3C1F3E5
:10952000A1C3C0F3F2D880ACFED7B3EF45F0A4C31B
:10953000A8F3A3C3A7F3A2C3A6F3A1C3A5F382A272
:10954000FED712000301AF6B030E0301AF5D0001F4
:1095500013E204EE15F00301AF51EB50BD6F0001B3
:10956000C0D845BE05D00301AE69AD690001120047
:109570000301AF2B0001E8E301EE98F020EC00F0CE
:109580000301AD6F1CC0AEF3000112000301BC6B00
:10959000BB6BBA6BB96BB76BB66BB56BB46BB86BB7
:1095A000000104EE1CF00301B851EB500B6E0B529E
:1095B0000001D8B479D004EE1CF00301B851EB508F
:1095C000BD6F00018ED845AE5AD0BCC329F0BBC3D5
:1095D00028F0BAC327F0B9C326F029C016F028C076
:1095E00015F027C014F026C013F01E6A1D6A1C6A0D
:1095F0000A0E1B6EB3EC02F016C029F015C028F05D
:1096000014C027F013C026F004EE1CF00301B8517B
:10961000EB500B6E2D6A2C6A2B6A0BC02AF00F0ED2
:109620002A142A6E000E2B142B6E000E2C142C6E96
:10963000000E2D142D6E2A502624B96F2B50272092
:10964000BA6F2C502820BB6F2D502920BC6F356A73
:10965000346A200E336E820E326EB7C339F0B6C351
:1096600038F0B5C337F0B4C336F068EC08F035C055
:10967000B7F334C0B6F333C0B5F332C0B4F300016E
:1096800004EE1CF00301B851EB500B6E2E0E0B5C78
:10969000000106E10301B76BB66BB56B7F0EB46FCB
:1096A0000301B82B00017CD7B7C339F0B6C338F03B
:1096B000B5C337F0B4C336F0BCC335F0BBC334F028
:1096C000BAC333F0B9C332F013EC09F002EC08F07E
:1096D00035C0B3F334C0B2F333C0B1F332C0B0F32A
:1096E0001200300E0301BD5D000ED8B0010E3B6EBE
:1096F0003A0EBD5D000102E3000E01D0010E3B16E3
:1097000002E0458E01D0459E1200010E0301BF5DAF
:1097100000010AE101EEFCF01F0EF76EDA0EF66EA4
:109720001FEC03F0EF6A23D001EEFCF01F0EF76E82
:10973000E80EF66E1FEC03F0EF6AC3C335F0C2C348
:1097400034F0C1C333F0C0C332F0396A386A480E0E
:10975000376E850E366EB8EC06F0010808E001EEB3
:10976000FCF0EE50FEE1ED52300EEE6EEF6AC3C338
:1097700035F0C2C334F0C1C333F0C0C332F0396A2C
:10978000386A200E376E820E366EB8EC06F001088D
:1097900008E001EEFCF0EE50FEE1ED52300EEE6E10
:1097A000EF6A01EEFCF0EE50FEE1ED52020E016EAA
:1097B000C3C329F0C2C328F0C1C327F0C0C326F039
:1097C000050EA7EC00F0EF6A45A809D00301BE051D
:1097D000FC0FE96E010EEA6AEA22200EEF6E00012C
:1097E000800E016E19EC00F001EEFCF0EE5003E08B
:1097F00043EC01F0FBD7200E43EC01F0030E43ECE9
:1098000001F0200E43EC01F0500E43EC01F0200E6D
:1098100043EC01F0020E43EC01F01F0EF76EF40E64
:10982000F66E3BEC01F0000E43EC01F0200E43EC31
:1098300001F0560E43EC01F0200E43EC01F0010E56
:0A98400043EC01F0200E43EF01F0AD
:020000040030CA
:03000100C81F1CF9
:02000500018177
:060008000FC00FE00F40E5
:0200000400F00A
:100000006C001800F80200006C00180068065AF82E
:10001000460484410F7E831E8FC5CC00FA00FF800A
:0400200025000000B7
:00000001FF
